:0300000002692C66
:10692C00758E1190000078FF79FFE4F0A3D9FBD8A5
:0D693C00F778FFE4F6D8FD75817F026984CD
:106D1F004401EA40490FDB4401E640C90FDB44015F
:056D2F00E23C8EFA3584
:0649DB009001CA12202821
:1049E1009001CEE0FCA3E0FDA3E0FEA3E0FFEF24F5
:1049F10069FFEE3474FEED34FFFDEC34FFFCEC1284
:104A01001B927BDF7A927986783D12196E9001D2E2
:104A11001220287B007A0079C078419001D2E0FC15
:104A2100A3E0FDA3E0FEA3E0FF121A771261987BD9
:104A3100007A0079C0784112196EC004C005C00621
:104A4100C0077F977E7E7DD57C409001D2E0F8A3A0
:104A5100E0F9A3E0FAA3E0FB12187DD003D002D065
:104A610001D000121879C004C005C006C0077F92AA
:104A71007E867DC07C419001CAE0F8A3E0F9A3E005
:104A8100FAA3E0FB12196EA804A905AA06AB07D088
:104A910007D006D005D00412187D9001DA12202823
:104AA1009001CEE0FCA3E0FDA3E0FEA3E0FFEF2434
:104AB10069FFEE3474FEED34FFFDEC34FFFCEC12C3
:104AC1001B929001CAE0F8A3E0F9A3E0FAA3E0FB8E
:104AD10012187D7B307AE67958783D12196EA80458
:104AE100A905AA06AB077F817E0E7DBA7C43121809
:104AF100799001E2E0F8A3E0F9A3E0FAA3E0FB1268
:104B0100196E9001D61220289001E6E0FCA3E0FD89
:104B1100A3E0FEA3E0FF9001D6E0F8A3E0F9A3E053
:104B2100FAA3E0FB121B14602940279001D6E0FC98
:104B3100A3E0FDA3E0FEA3E0FF9001E6E0F8A3E01F
:104B4100F9A3E0FAA3E0FB1218799001D61220280C
:104B510080B69001E6E0FCA3E0FDA3E0FEA3E0FF48
:104B6100121B819001D6E0F8A3E0F9A3E0FAA3E0DB
:104B7100FB121B1450279001D6E0FCA3E0FDA3E03B
:104B8100FEA3E0FF9001E6E0F8A3E0F9A3E0FAA3B9
:104B9100E0FB12187D9001D612202880B57F007E9F
:104BA100007D007C009001D6E0F8A3E0F9A3E0FAD3
:104BB100A3E0FB121B14604840469001EAE0FCA30D
:104BC100E0FDA3E0FEA3E0FF9001D6E0F8A3E0F949
:104BD100A3E0FAA3E0FB121B1450259001D6E0FCE0
:104BE100A3E0FDA3E0FEA3E0FF9001E6E0F8A3E06F
:104BF100F9A3E0FAA3E0FB1218799001D61220285C
:104C01007F007E007D007C009001D6E0F8A3E0F9F2
:104C1100A3E0FAA3E0FB121B14504B9001EAE0FC65
:104C2100A3E0FDA3E0FEA3E0FF121B819001D6E00B
:104C3100F8A3E0F9A3E0FAA3E0FB121B14602740FC
:104C4100259001D6E0FCA3E0FDA3E0FEA3E0FF90E8
:104C510001E6E0F8A3E0F9A3E0FAA3E0FB12187D76
:104C61009001D61220289001D6E0FCA3E0FDA3E03C
:104C7100FEA3E0FF1259FE7B247A0B799878391252
:104C8100196E9001DAE0F8A3E0F9A3E0FAA3E0FBE2
:104C910012187D9001DE1220287B007A0079C078FD
:104CA100419001DEE0FCA3E0FDA3E0FEA3E0FF12E2
:104CB1001A771261987B007A0079C0784112196ED7
:104CC100A804A905AA06AB079001DEE0FCA3E0FD5C
:094CD100A3E0FEA3E0FF12187934
:014CDA0022B7
:106DAC009001F51220289001F5E0FCA3E0FDA3E092
:106DBC00FEA3E0FF126198A804A905AA06AB0790F0
:106DCC0001F5E0FCA3E0FDA3E0FEA3E0FF121879BF
:106DDC009001E6E0F8A3E0F9A3E0FAA3E0FB1219B6
:026DEC006E2215
:060D470090015A12202861
:100D4D0090015AE0FCA3E0FDA3E0FEA3E0FFEF2439
:100D5D0013FFEE342DFEED34FFFDEC34FFFCEC12F1
:100D6D001B9290015EE0F8A3E0F9A3E0FAA3E0FB8B
:100D7D0012187D9001621220287F8D7EA67D147C35
:100D8D003D900162E0F8A3E0F9A3E0FAA3E0FB12C5
:100D9D00196E7B807AF279BF783E12187D126DAC98
:100DAD009001661220287F477E857D167C3D90013F
:100DBD0062E0F8A3E0F9A3E0FAA3E0FB12196E7B61
:100DCD00937AA77984783E12187D126DAC90016AE2
:100DDD001220287F217EB47D0A7C3D900162E0F8CF
:100DED00A3E0F9A3E0FAA3E0FB12196E7BFF7ACD25
:100DFD007953783F12187D126DAC90016E12202838
:100E0D007F4D7E6C7D337C3B900162E0F8A3E0F971
:100E1D00A3E0FAA3E0FB12196E7B817A3D797E780F
:100E2D003F12187D126DAC9001721220287F007E4A
:100E3D00007D007C4090016EE0F8A3E0F9A3E0FA9C
:100E4D00A3E0FB12196EA804A905AA06AB07900131
:100E5D0066E0FCA3E0FDA3E0FEA3E0FF121879120B
:100E6D0059E87BF37A767914783F12196EC004C075
:100E7D0005C006C007900166E0FCA3E0FDA3E0FEFF
:100E8D00A3E0FF1259E87BE87AC179517840121935
:100E9D006EA804A905AA06AB077FB17E737D717C90
:100EAD0042121879D003D002D001D000121879C0A7
:100EBD0004C005C006C0077F007E007D007C409009
:100ECD00016EE0F8A3E0F9A3E0FAA3E0FB12196EBE
:100EDD001259E87B0C7A5979ED783E12196EA804F7
:100EED00A905AA06AB07D007D006D005D004121865
:100EFD00799001761220287F007E007D007C409045
:100F0D00016EE0F8A3E0F9A3E0FAA3E0FB12196E7D
:100F1D00C004C005C006C0077F007E007D007C4078
:100F2D00900166E0F8A3E0F9A3E0FAA3E0FB121943
:100F3D006ED003D002D001D0001218791259E87B7F
:100F4D00767A4F791E783D12196EC004C005C00621
:100F5D00C0077F007E007D007C40900166E0F8A315
:100F6D00E0F9A3E0FAA3E0FB12196E1259E87B9C9D
:100F7D007A5A79B6783D12196EA804A905AA06AB5E
:100F8D0007900176E0FCA3E0FDA3E0FEA3E0FF12D5
:100F9D001879A804A905AA06AB07D007D006D00575
:100FAD00D00412187DC004C005C006C0077F007EA6
:100FBD00007D007C4090016EE0F8A3E0F9A3E0FA1B
:100FCD00A3E0FB12196E900172E0F8A3E0F9A3E023
:100FDD00FAA3E0FB1218791259E87B687A96790426
:100FED00783D12196EA804A905AA06AB07D007D043
:100FFD0006D005D0041218799001761220287F00B2
:10100D007E007D007C4090016EE0F8A3E0F9A3E046
:10101D00FAA3E0FB12196EA804A905AA06AB079066
:10102D000166E0FCA3E0FDA3E0FEA3E0FF1218794A
:10103D00900172E0F8A3E0F9A3E0FAA3E0FB121827
:10104D007D1259E87BD87A2A79C1783C12196EC085
:10105D0004C005C006C0077F007E007D007C409067
:10106D00016EE0F8A3E0F9A3E0FAA3E0FB12196E1C
:10107D00A804A905AA06AB07900166E0FCA3E0FD54
:10108D00A3E0FEA3E0FF1218791259E87B727A33C0
:10109D0079DC783C12196EA804A905AA06AB079055
:1010AD000176E0FCA3E0FDA3E0FEA3E0FF121879BA
:1010BD00D003D002D001D000121879C004C005C0F1
:1010CD0006C007900172E0F8A3E0F9A3E0FAA3E0EF
:1010DD00FB900166E0FCA3E0FDA3E0FEA3E0FF12A0
:1010ED0018791259E87B307A4C79A6783C12196E32
:1010FD00A804A905AA06AB07D007D006D005D004D1
:10110D0012187990017612202890016EE0FCA3E070
:10111D00FDA3E0FEA3E0FF1259E87B0B7AD2798C98
:10112D00783C12196E900176E0F8A3E0F9A3E0FA8D
:10113D00A3E0FB12187DC004C005C006C0079001D6
:10114D0072E0FCA3E0FDA3E0FEA3E0FF900166E0EA
:10115D00F8A3E0F9A3E0FAA3E0FB12187D1259E819
:10116D007B697AE37988783C12196EA804A905AADF
:10117D0006AB07D007D006D005D00412187D90011C
:10118D00761220287F007E007D007C4090016AE071
:10119D00F8A3E0F9A3E0FAA3E0FB12196EA804A9E5
:1011AD0005AA06AB07900166E0FCA3E0FDA3E0FEF7
:1011BD00A3E0FF1218791259E87BF97A4E794C7831
:1011CD003C12196EC004C005C006C007900172E044
:1011DD00FCA3E0FDA3E0FEA3E0FF1259E87BCD7A6E
:1011ED00AF79E6783B12196EA804A905AA06AB07DC
:1011FD00D007D006D005D00412187DC004C005C09C
:10120D0006C0077F007E007D007C4090016EE0F8F7
:10121D00A3E0F9A3E0FAA3E0FB12196E900172E0CE
:10122D00F8A3E0F9A3E0FAA3E0FB12187D1259E848
:10123D007BBC7A5779AD783B12196EA804A905AA23
:10124D0006AB07D007D006D005D00412187DC00418
:10125D00C005C006C0077F007E007D807C409001E8
:10126D006EE0F8A3E0F9A3E0FAA3E0FB12196EA873
:10127D0004A905AA06AB07900166E0FCA3E0FDA357
:10128D00E0FEA3E0FF1218791259E87B4E7AB4798B
:10129D00AB783B12196EA804A905AA06AB07D007B7
:1012AD00D006D005D00412187990017A1220287F2B
:1012BD00007E007D007C4090016EE0F8A3E0F9A374
:1012CD00E0FAA3E0FB12196EA804A905AA06AB0764
:1012DD00900166E0FCA3E0FDA3E0FEA3E0FF121881
:1012ED0079900172E0F8A3E0F9A3E0FAA3E0FB1214
:1012FD0018791259E87BA97A6A7982783B12196EAE
:10130D0090017AE0F8A3E0F9A3E0FAA3E0FB12184C
:10131D007DC004C005C006C0077F007E007D407CF7
:10132D0040900166E0F8A3E0F9A3E0FAA3E0FB1218
:10133D00196E1259E87B9C7ADC796F783B12196E25
:10134D00A804A905AA06AB07D007D006D005D0047E
:10135D00121879C004C005C006C0077F007E007D4D
:10136D00807C4090016EE0F8A3E0F9A3E0FAA3E0E1
:10137D00FB12196EC004C005C006C0077F007E00B9
:10138D007D007C40900166E0F8A3E0F9A3E0FAA3AC
:10139D00E0FB12196ED003D002D001D000121879E3
:1013AD001259E87BCA7A547941783B12196EA80418
:1013BD00A905AA06AB07D007D006D005D004121890
:1013CD007990017A1220287F007E007D007C40906C
:1013DD00016EE0F8A3E0F9A3E0FAA3E0FB12196EA9
:1013ED00C004C005C006C0077F007E007D407C4064
:1013FD00900166E0F8A3E0F9A3E0FAA3E0FB12196F
:10140D006ED003D002D001D0001218791259E87BAA
:10141D00457A2F7923783B12196EC004C005C0069A
:10142D00C007900172E0FCA3E0FDA3E0FEA3E0FF86
:10143D0090016EE0F8A3E0F9A3E0FAA3E0FB121827
:10144D007D1259E87B147A5C792C783B12196EA8C1
:10145D0004A905AA06AB0790017AE0FCA3E0FDA361
:10146D00E0FEA3E0FF121879A804A905AA06AB07B0
:10147D00D007D006D005D00412187DC004C005C019
:10148D0006C0077F007E007D007C4090016EE0F875
:10149D00A3E0F9A3E0FAA3E0FB12196E900166E058
:1014AD00F8A3E0F9A3E0FAA3E0FB12187D90017216
:1014BD00E0F8A3E0F9A3E0FAA3E0FB1218791259C2
:1014CD00E87BA67AD57910783B12196EA804A90588
:1014DD00AA06AB07D007D006D005D004121879C0E4
:1014ED0004C005C006C0077F007E007D007C4090D3
:1014FD00016EE0F8A3E0F9A3E0FAA3E0FB12196E88
:10150D00C004C005C006C0077F007E007D007C4082
:10151D0090016AE0F8A3E0F9A3E0FAA3E0FB121949
:10152D006ED003D002D001D0001218791259E87B89
:10153D00B37A7B79F2783A12196EA804A905AA0636
:10154D00AB07D007D006D005D00412187D90017AD4
:10155D001220287F007E007D007C4090016AE0F81B
:10156D00A3E0F9A3E0FAA3E0FB12196E900166E087
:10157D00F8A3E0F9A3E0FAA3E0FB12187DC004C0C4
:10158D0005C006C0077F007E007D007C4090016E87
:10159D00E0F8A3E0F9A3E0FAA3E0FB12196EA804AA
:1015AD00A905AA06AB07D007D006D005D00412189E
:1015BD00791259E87B047AAD79C0783A12196EC068
:1015CD0004C005C006C0077F007E007D007C4090F2
:1015DD000172E0F8A3E0F9A3E0FAA3E0FB12196EA3
:1015ED00C004C005C006C0077F007E007D007C40A2
:1015FD0090016EE0F8A3E0F9A3E0FAA3E0FB121965
:10160D006ED003D002D001D0001218791259E87BA8
:10161D00A37A0679D378BA12196EA804A905AA0679
:10162D00AB07D007D006D005D00412187DC004C07A
:10163D0005C006C0077F007E007D807C4090016E56
:10164D00E0F8A3E0F9A3E0FAA3E0FB12196E12593A
:10165D00E87B4B7A1F79BA783A12196EA804A9055E
:10166D00AA06AB07D007D006D005D004121879C052
:10167D0004C005C006C0077F007E007D007C409041
:10168D00016EE0F8A3E0F9A3E0FAA3E0FB12196EF6
:10169D00C004C005C006C0077F007E007D007C40F1
:1016AD00900166E0F8A3E0F9A3E0FAA3E0FB1219BC
:1016BD006ED003D002D001D000121879900172E0E3
:1016CD00F8A3E0F9A3E0FAA3E0FB12187D1259E8A4
:1016DD007BA97A3079B6783A12196EA804A905AAB1
:1016ED0006AB07D007D006D005D00412187D9001A7
:1016FD007E1220287F007E007D807C4090016EE070
:10170D00F8A3E0F9A3E0FAA3E0FB12196EA804A96F
:10171D0005AA06AB07900166E0FCA3E0FDA3E0FE81
:10172D00A3E0FF121879900172E0F8A3E0F9A3E0AD
:10173D00FAA3E0FB12187D1259E87B3B7AAA799A3D
:10174D00783A12196EA804A905AA06AB0790017E76
:10175D00E0FCA3E0FDA3E0FEA3E0FF121879C004B6
:10176D00C005C006C0077F007E007D007C40900153
:10177D006EE0F8A3E0F9A3E0FAA3E0FB12196EC046
:10178D0004C005C006C0077F007E007D007C409030
:10179D000166E0F8A3E0F9A3E0FAA3E0FB12196EED
:1017AD00A804A905AA06AB07D007D006D005D0041A
:1017BD0012187D1259E87B247A0B7998783A121910
:1017CD006EA804A905AA06AB07D007D006D005D090
:1017DD0004121879C004C005C006C0077F007E0042
:1017ED007D007C40900166E0F8A3E0F9A3E0FAA348
:1017FD00E0FB12196E900172E0F8A3E0F9A3E0FA94
:10180D00A3E0FB1218791259E87BE07A2D799078D4
:10181D003A12196EA804A905AA06AB07D007D0067F
:10182D00D005D00412187990017E12202890017AEB
:10183D00E0FCA3E0FDA3E0FEA3E0FF900176E0F85D
:10184D00A3E0F9A3E0FAA3E0FB12187D90017EE07E
:10185D00F8A3E0F9A3E0FAA3E0FB12187D7B487A28
:08186D005179C7784512196E8C
:011875002250
:0B2B2F00900120EBF0A3EAF0A3E9F016
:102B3A00900126E0FCA3E0FDA3E0FEA3E0FFEC1277
:102B4A001B927B007A81798878C612187D90012AB7
:102B5A00E0F8A3E0F9A3E0FAA3E0FB12187D9001E4
:102B6A002E1220287F0A7EEB7D157C3D90012EE0F7
:102B7A00F8A3E0F9A3E0FAA3E0FB12196E7B7F7ACF
:102B8A004F7940783F12187D126DAC9001321220B5
:102B9A00287F8C7EA67D147C3D90012EE0F8A3E070
:102BAA00F9A3E0FAA3E0FB12196E7B367A90795208
:102BBA00783F12187D126DAC9001361220287F4D95
:102BCA007E6C7D337C3B90012EE0F8A3E0F9A3E014
:102BDA00FAA3E0FB12196E7B857AEA797E783F12B6
:102BEA00187D126DAC90013A1220287F217EB47DA7
:102BFA000A7C3D90012EE0F8A3E0F9A3E0FAA3E0F5
:102C0A00FB12196E7BD37A697979783F12187D1293
:102C1A006DAC90013E1220287F477E857D167C3D53
:102C2A0090012EE0F8A3E0F9A3E0FAA3E0FB121961
:102C3A006E7B9F7A027900783D12187D126DAC90F6
:102C4A0001421220287F007E007D007C4090013ED8
:102C5A00E0F8A3E0F9A3E0FAA3E0FB12196E125917
:102C6A00FE7BB07A727928783F12196EC004C005CB
:102C7A00C006C007900136E0FCA3E0FDA3E0FEA376
:102C8A00E0FF1259FE7B7D7A3F79C9784012196EAE
:102C9A00A804A905AA06AB07D007D006D005D00418
:102CAA0012187DC004C005C006C0077F007E007DE3
:102CBA00007C4090013EE0F8A3E0F9A3E0FAA3E02B
:102CCA00FB12196EA804A905AA06AB07900136E003
:102CDA00FCA3E0FDA3E0FEA3E0FF1218791259FE5F
:102CEA007B6F7A1279A3783F12196EA804A905AAF4
:102CFA0006AB07D007D006D005D004121879C00455
:102D0A00C005C006C00790013AE0FCA3E0FDA3E0BD
:102D1A00FEA3E0FF1259FE7BC97A76793E783E120D
:102D2A00196EA804A905AA06AB07D007D006D005D4
:102D3A00D0041218799001E2E0F8A3E0F9A3E0FACE
:102D4A00A3E0FB12196E900132E0F8A3E0F9A3E0C8
:102D5A00FAA3E0FB12187D90014612202890014642
:102D6A00E0FCA3E0FDA3E0FEA3E0FFC004C005C0B1
:102D7A0006C0077F007E007D007C40900142E0F89B
:102D8A00A3E0F9A3E0FAA3E0FB12196E1259FE7B45
:102D9A00D57A7879E9783D12196EC004C005C00663
:102DAA00C0077F007E007D007C40900136E0F8A3DA
:102DBA00E0F9A3E0FAA3E0FB12196E1259FE7BD1E7
:102DCA007A22795B783E12196ED003D002D001D0F4
:102DDA0000121879C004C005C006C0077F007E0033
:102DEA007D007C4090013EE0F8A3E0F9A3E0FAA35D
:102DFA00E0FB12196EC004C005C006C0077F007E42
:102E0A00007D007C40900136E0F8A3E0F9A3E0FAE7
:102E1A00A3E0FB12196ED003D002D001D000121821
:102E2A00791259FE7BFC7AA97971783D12196EA83C
:102E3A0004A905AA06AB07D007D006D005D004120C
:102E4A001879C004C005C006C0077F007E007D0057
:102E5A007C4090013EE0F8A3E0F9A3E0FAA3E0FB8E
:102E6A0012196EC004C005C006C00790013AE0FC02
:102E7A00A3E0FDA3E0FEA3E0FF900136E0F8A3E0A3
:102E8A00F9A3E0FAA3E0FB12187DD003D002D00127
:102E9A00D0001218791259FE7BD57A787969783D73
:102EAA0012196EA804A905AA06AB07D007D006D046
:102EBA0005D0041218799001E2E0F8A3E0F9A3E042
:102ECA00FAA3E0FB12196EA804A905AA06AB07D05B
:102EDA0007D006D005D00412187D9001461220288A
:102EEA007F007E007D007C4090013EE0F8A3E0F97F
:102EFA00A3E0FAA3E0FB12196E1259FE7BE37AC72C
:102F0A007928783F12196EC004C005C006C0079020
:102F1A000136E0FCA3E0FDA3E0FEA3E0FF1259FEA8
:102F2A007B9E7A5E79C7784012196EA804A905AA11
:102F3A0006AB07D007D006D005D00412187DC0040E
:102F4A00C005C006C0077F007E007D007C4090015E
:102F5A003EE0F8A3E0F9A3E0FAA3E0FB12196EA899
:102F6A0004A905AA06AB07900136E0FCA3E0FDA37D
:102F7A00E0FEA3E0FF1218791259FE7BE57AD079B8
:102F8A00A2783F12196EA804A905AA06AB07D007B2
:102F9A00D006D005D0041218799001E2E0F8A3E037
:102FAA00F9A3E0FAA3E0FB12196E900142E0F8A33C
:102FBA00E0F9A3E0FAA3E0FB12187D90014A12207F
:102FCA00287F007E007D007C4090013EE0F8A3E06F
:102FDA00F9A3E0FAA3E0FB12196EA804A905AA0650
:102FEA00AB07900142E0FCA3E0FDA3E0FEA3E0FFF3
:102FFA001218791259FE7B067A817915783E1219D0
:10300A006EC004C005C006C00790014AE0FCA3E0F8
:10301A00FDA3E0FEA3E0FF1259FE7BA67A9B79A4EA
:10302A00784012196ED003D002D001D0001218795C
:10303A009001E2E0F8A3E0F9A3E0FAA3E0FB121999
:10304A006E90014E122028900146E0FCA3E0FDA3F9
:10305A00E0FEA3E0FF1259FEC004C005C006C00787
:10306A0090014EE0FCA3E0FDA3E0FEA3E0FF1259AD
:10307A00E8A804A905AA06AB07D007D006D005D050
:10308A000412196E7B327AAF79CB783E12196EC070
:10309A0004C005C006C00790014EE0FCA3E0FDA3F2
:1030AA00E0FEA3E0FF1259FE7BDB7ADE796A783F05
:1030BA0012196EA804A905AA06AB07D007D006D034
:1030CA0005D00412187D900123E0FBA3E0FAA3E0E7
:1030DA00F9121FB6900123E0FBA3E0FAA3E0F9126C
:1030EA001F96900123E0FBA3E0FAA3E0F91220085F
:1030FA0012196EA804A905AA06AB077F007E007DF7
:10310A00807C3F12187912673D9000E812202890BF
:10311A000123E0FBA3E0FAA3E0F9121F961269C9A2
:10312A00900123E0FBA3E0FAA3E0F9121FB6900195
:10313A0046E0FCA3E0FDA3E0FEA3E0FF1259E8C0CD
:10314A0004C005C006C00790014EE0FCA3E0FDA341
:10315A00E0FEA3E0FF1259E8A804A905AA06AB07F6
:10316A00D007D006D005D00412196EC004C005C01D
:10317A0006C007900123E0FBA3E0FAA3E0F9121FBF
:10318A00961259E8A804A905AA06AB07D007D006E3
:10319A00D005D004121A77900152122028900146C5
:1031AA00E0FCA3E0FDA3E0FEA3E0FF1259FEC00489
:1031BA00C005C006C00790014EE0FCA3E0FDA3E0F5
:1031CA00FEA3E0FF1259E8A804A905AA06AB07D096
:1031DA0007D006D005D00412196E7BDB7ADE796A35
:1031EA00783F12196EC004C005C006C00790014E90
:1031FA00E0FCA3E0FDA3E0FEA3E0FF1259FE7B3250
:10320A007AAF79CB783E12196EA804A905AA06AB43
:10321A0007D007D006D005D004121879C004C0051B
:10322A00C006C007900123E0FBA3E0FAA3E0F9126D
:10323A001F961259E8A804A905AA06AB07D007D019
:10324A0006D005D004121A77900156122028900150
:10325A0056E0FCA3E0FDA3E0FEA3E0FFC004C00526
:10326A00C006C007900152E0FCA3E0FDA3E0FEA364
:10327A00E0FF9000E8122028D007D006D005D0043D
:10328A001269C9900120E0FBA3E0FAA3E0F9121F3A
:10329A00B6900120E0FBA3E0FAA3E0F9121F967BA7
:1032AA00007A0079007800121B146030402E9001D9
:1032BA0020E0FBA3E0FAA3E0F9C003C002C00112B8
:1032CA001F969001E6E0F8A3E0F9A3E0FAA3E0FB79
:1032DA0012187DD001D002D003121FB6900120E04F
:1032EA00FBA3E0FAA3E0F9121F969001E6E0F8A327
:1032FA00E0F9A3E0FAA3E0FB121B14502E90012080
:10330A00E0FBA3E0FAA3E0F9C003C002C001121F68
:10331A00969001E6E0F8A3E0F9A3E0FAA3E0FB1235
:0B332A001879D001D002D003121FB6AA
:013335002275
:0B4613009001A8EBF0A3EAF0A3E9F08F
:10461E009001AEE0FCA3E0FDA3E0FEA3E0FFEC12F0
:10462E001B927B007A81798878C612187D9001B230
:10463E00E0F8A3E0F9A3E0FAA3E0FB12187D7B00FB
:10464E007AAD790E7847121A779001B61220287F2C
:10465E00A67EFE7DC77C429001B6E0F8A3E0F9A3EA
:10466E00E0FAA3E0FB12196E7B917AEA797E783F2D
:10467E0012187D126DAC9001BA1220287F117E2384
:10468E007D5F7C379001B6E0F8A3E0F9A3E0FAA3D2
:10469E00E0FB12196EA804A905AA06AB077F507E8F
:1046AE00AC7DAE7C3B121879126DACC004C005C057
:1046BE0006C0079001BAE0FCA3E0FDA3E0FEA3E074
:1046CE00FF1259FEA804A905AA06AB07D007D0060B
:1046DE00D005D00412196EC004C005C006C0077FF5
:1046EE00187E017DC87C429001B6E0F8A3E0F9A3E4
:1046FE00E0FAA3E0FB12196E7B327AE47946783F3A
:10470E0012187D126DACA804A905AA06AB07D00736
:10471E00D006D005D00412187DC004C005C006C056
:10472E00077F007E007D007C409001BAE0F8A3E098
:10473E00F9A3E0FAA3E0FB12196E1259FE7B0C7A74
:10474E00347969783812196EA804A905AA06AB0740
:10475E00D007D006D005D00412187D9001BE1220CD
:10476E00287F147E6A7D177C389001B6E0F8A3E0AE
:10477E00F9A3E0FAA3E0FB12196EA804A905AA0694
:10478E00AB077F6D7E6A7D857C3D121879126DAC0C
:10479E009001C21220289001BEE0FCA3E0FDA3E030
:1047AE00FEA3E0FF125A3AC004C005C006C007902F
:1047BE0001C2E0FCA3E0FDA3E0FEA3E0FF1259E876
:1047CE00A804A905AA06AB07D007D006D005D004C9
:1047DE0012196E125B489001A8E0FBA3E0FAA3E069
:1047EE00F9121FB69001E6E0F8A3E0F9A3E0FAA3F0
:1047FE00E0FB9001BEE0FCA3E0FDA3E0FEA3E0FF22
:10480E00121A771261989001E6E0F8A3E0F9A3E09E
:10481E00FAA3E0FB12196EA804A905AA06AB07902D
:10482E0001BEE0FCA3E0FDA3E0FEA3E0FF121879B9
:10483E009001C61220287F007E007DC07C3F900133
:10484E00EAE0F8A3E0F9A3E0FAA3E0FB12196E90F8
:10485E0001C6E0F8A3E0F9A3E0FAA3E0FB121B14F3
:10486E00505A7F007E007D007C3F9001EAE0F8A365
:10487E00E0F9A3E0FAA3E0FB12196E9001C6E0F88E
:10488E00A3E0F9A3E0FAA3E0FB121B14402E900163
:10489E00A8E0FBA3E0FAA3E0F9C003C002C0011236
:1048AE001F969001EAE0F8A3E0F9A3E0FAA3E0FB7B
:1048BE0012187DD001D002D003121FB69001A8E0CD
:1048CE00FBA3E0FAA3E0F9C003C002C001121F96D9
:1048DE00C004C005C006C0079001A8E0FBA3E0FA23
:1048EE00A3E0F9121F969001E6E0F8A3E0F9A3E029
:1048FE00FAA3E0FB121A771261989001E6E0F8A392
:10490E00E0F9A3E0FAA3E0FB12196EA804A905AA28
:10491E0006AB07D007D006D005D004121879D00107
:10492E00D002D003121FB69001BEE0FCA3E0FDA39F
:10493E00E0FEA3E0FF1259FEC004C005C006C0078A
:10494E009001C2E0FCA3E0FDA3E0FEA3E0FF12593C
:10495E00FEA804A905AA06AB07D007D006D005D03D
:10496E000412196E9001ABE0FBA3E0FAA3E0F9127A
:10497E001FB69001ABE0FBA3E0FAA3E0F9121F967D
:10498E009001ABE0FBA3E0FAA3E0F91220081219A4
:10499E006EA804A905AA06AB077F007E007D807C69
:1049AE003F12187912673D9000E81220289001AB53
:1049BE00E0FBA3E0FAA3E0F9121F961269C9900179
:0C49CE00ABE0FBA3E0FAA3E0F9121FB677
:0149DA0022BA
:0B333600900182EBF0A3EAF0A3E9F0A5
:103341007F927E0A7D867C3E900188E0F8A3E0F9B9
:10335100A3E0FAA3E0FB12196E90018CE0F8A3E060
:10336100F9A3E0FAA3E0FB12187990019412202846
:103371007F007E007D007C00900194E0F8A3E0F9DD
:10338100A3E0FAA3E0FB121B145027900194E0FC88
:10339100A3E0FDA3E0FEA3E0FF9001E6E0F8A3E0D7
:1033A100F9A3E0FAA3E0FB12187D90019412202802
:1033B10080489001E6E0FCA3E0FDA3E0FEA3E0FF6E
:1033C100900194E0F8A3E0F9A3E0FAA3E0FB121B5B
:1033D1001460274025900194E0FCA3E0FDA3E0FEEA
:1033E100A3E0FF9001E6E0F8A3E0F9A3E0FAA3E08F
:1033F100FB121879900194122028900194E0F8A30F
:10340100E0F9A3E0FAA3E0FB90001EE0FCA3E0FDDD
:10341100A3E0FEA3E0FF1218799000161220289075
:103421000016E0FCA3E0FDA3E0FEA3E0FF1259E8D3
:10343100C004C005C006C00790001AE0FCA3E0FD6F
:10344100A3E0FEA3E0FF1259E8A804A905AA06AB70
:1034510007D007D006D005D00412196EC004C005EC
:10346100C006C007900190E0FCA3E0FDA3E0FEA32D
:10347100E0FF1259E8A804A905AA06AB07D007D0B6
:1034810006D005D00412196EC004C005C006C007DD
:1034910090001AE0FCA3E0FDA3E0FEA3E0FF1259B7
:1034A100FEC004C005C006C007900190E0FCA3E087
:1034B100FDA3E0FEA3E0FF1259FEA804A905AA0698
:1034C100AB07D007D006D005D00412196EA804A905
:1034D10005AA06AB07D007D006D005D00412187D87
:1034E100900198122028900198E0FCA3E0FDA3E050
:1034F100FEA3E0FF900198E0F8A3E0F9A3E0FAA3AE
:10350100E0FB12196EA804A905AA06AB077F007E8D
:10351100007D807C3F12187912673D90019C12203A
:1035210028900198E0FCA3E0FDA3E0FEA3E0FFC02A
:1035310004C005C006C00790019CE0FCA3E0FDA308
:10354100E0FEA3E0FF9000E8122028D007D006D0CB
:1035510005D0041269C9900185E0FBA3E0FAA3E05C
:10356100F9121FB6900185E0FBA3E0FAA3E0F9127E
:103571001F961259E8C004C005C006C00790018516
:10358100E0FBA3E0FAA3E0F9121F961259FED00363
:10359100D002D001D000121A77C004C005C006C005
:1035A1000790001AE0FCA3E0FDA3E0FEA3E0FF12F8
:1035B10059E8C004C005C006C00790001AE0FCA38A
:1035C100E0FDA3E0FEA3E0FF1259FED003D002D03C
:1035D10001D000121A77A804A905AA06AB07D007E3
:1035E100D006D005D00412196EC004C005C006C0B3
:1035F10007900185E0FBA3E0FAA3E0F9121F961200
:1036010059E8C004C005C006C00790001AE0FCA339
:10361100E0FDA3E0FEA3E0FF1259E8A804A905AA72
:1036210006AB07D007D006D005D00412196EC0042E
:10363100C005C006C007900190E0FCA3E0FDA3E037
:10364100FEA3E0FF1259FED003D002D001D0001238
:103651001A77D003D002D001D0001218799001A4BA
:10366100122028900190E0FCA3E0FDA3E0FEA3E07E
:10367100FF1259E8C004C005C006C00790001AE057
:10368100FCA3E0FDA3E0FEA3E0FF1259E8A804A912
:1036910005AA06AB07D007D006D005D00412196ED3
:1036A100C004C005C006C007900016E0FCA3E0FD01
:1036B100A3E0FEA3E0FF1259E8A804A905AA06ABFE
:1036C10007D007D006D005D00412196EC004C0057A
:1036D100C006C007900190E0FCA3E0FDA3E0FEA3BB
:1036E100E0FF1259FEC004C005C006C00790001AD1
:1036F100E0FCA3E0FDA3E0FEA3E0FF1259FEA80455
:10370100A905AA06AB07D007D006D005D004121927
:103711006EA804A905AA06AB07D007D006D005D02C
:103721000412187D9001A0122028900190E0FCA3C2
:10373100E0FDA3E0FEA3E0FF1259E8C004C005C00C
:1037410006C007900016E0FCA3E0FDA3E0FEA3E0A5
:10375100FF1259FEA804A905AA06AB07D007D00697
:10376100D005D00412196EC004C005C006C0079070
:1037710001A0E0FCA3E0FDA3E0FEA3E0FF9001A017
:10378100E0F8A3E0F9A3E0FAA3E0FB12196EA804A4
:10379100A905AA06AB077F007E007D807C3F121839
:1037A1007912673DA804A905AA06AB07D007D00680
:1037B100D005D004121A779001A01220289001A000
:1037C100E0FCA3E0FDA3E0FEA3E0FFC004C005C050
:1037D10006C0079001A4E0FCA3E0FDA3E0FEA3E086
:1037E100FF9000E8122028D007D006D005D004129F
:1037F10069C9900182E0FBA3E0FAA3E0F9121FB6C8
:10380100900182E0FBA3E0FAA3E0F9121F967B008E
:103811007A0079007800121B146030402E900182EA
:10382100E0FBA3E0FAA3E0F9C003C002C001121F4C
:10383100969001E6E0F8A3E0F9A3E0FAA3E0FB1219
:0B384100187DD001D002D003121FB68A
:01384C002259
:10668D00323B171C0205006400640001000007A3E3
:10669D0000870384006407080384068205690007E8
:1066AD0000020009003B003B0017001C000C0063BA
:1066BD0000C700C70002000A0E0F03840E0F0384EB
:1066CD000E0F07080E0F070800080007000E000048
:1066DD0000000000000100010000000100010000A9
:1066ED00000000000000000000000000000000009D
:1066FD000000000000000000000000030000000387
:10670D000002000300020003000300020003000268
:10671D00000300000003000100030002000300025B
:0C672D0000030003000200030002000350
:066D3400C119C11BC11AC8
:106B00009000107432F0900011743BF090001274F9
:106B100017F0900013741CF09000147402F09000B1
:106B2000157405F0124FD5757900757A00D3E57AA2
:106B3000940EE57964809480503CE57A25E0FFE589
:106B40007933FE74932FF58274663EF583E493FCEB
:106B5000740193FDE57A25E0FFE57933FE74222F79
:106B6000F58274003EF583ECF0A3EDF0057AE57A4A
:106B70007002057980B71250D9900068E4F0A3E460
:106B8000F090006AE4F0A3E4F090006CE4F0A3E479
:056B9000F01250FB2291
:1041C80090003FE0F574D3E57464809482400BC39B
:1041D800E574648094865002C219E5A064FFFFEF7D
:1041E8005407F576E5766006C29CC2988002D29C98
:1041F800E5765406FFEF60270578E578D3940A4002
:104208000F75750AC3E57464809486500375780A3F
:10421800E578D39414400E75756475781480067526
:104228007800757501AF74EF3395E0FEEF25E0FF78
:10423800EE33FE74DB2FF58274663EF583E493F566
:1042480072740193F573AF74EF3395E0FEEF25E0D8
:10425800FFEE33FE74B12FF58274663EF583E49366
:10426800F570740193F571E5746403706B90001533
:10427800E0FFEF75F004121E50AFF0EF602E9000D3
:1042880014E0FFEF3395E0FEEF25E0FFEE33FE7418
:10429800052FF58274673EF583E493FE740193FF5E
:1042A800EF2571F571EE3570F570802C900014E0F3
:1042B800FFEF3395E0FEEF25E0FFEE33FE741F2F8E
:1042C800F58274673EF583E493FE740193FFEF254E
:1042D80071F571EE3570F570E576B401109000282F
:1042E800E0FEA3E0FFEF4E700405778003757700CA
:1042F800E577C394144008757700A219B39219D3CF
:10430800E5766480948150030245B7C3E574648000
:10431800948640030243DD12502AE5766404705502
:10432800AF74EF3395E0FE74102FF58274003EF5FC
:1043380083E02575F0AF74EF3395E0FE74102FF528
:104348008274003EF583E0FFEF3395E0FED3EF95EE
:1043580071E5706480F8EE6480984016AF73AE74AF
:10436800EEFD3395E0FC74102DF58274003CF58366
:10437800EFF0124FD5E5766402705AAF74EF3395BB
:10438800E0FE74102FF58274003EF583E0FFC3EF62
:104398009575FFEFF0AF74EF3395E0FE74102FF5CD
:1043A8008274003EF583E0FFEF3395E0FEC3EF959E
:1043B80073E5726480F8EE6480985016AF71AE743D
:1043C800EEFD3395E0FC74102DF58274003CF58306
:1043D800EFF0124FD5C3E57464809486500302440D
:1043E800F974FA2574F574E57664047072AF75EFA4
:1043F800FD7C00AF74EF3395E0FEEF25E0FFEE3370
:10440800FE74222FF58274003EF583EC8DF0121FA6
:1044180012AF74EF3395E0FEEF25E0FFEE33FE7444
:10442800222FF58274003EF583E0FEA3E0FFD3EF70
:104438009571E5706480F8EE648098401FAF74EF62
:104448003395E0FEEF25E0FFEE33FE74222FF58270
:1044580074003EF583E572F0A3E573F01250D9E5D8
:1044680076640260030244F3AF74EF3395E0FEEF25
:1044780025E0FFEE33FE74222FF58274003EF583AB
:10448800C083C082E0FEA3E0FFAD757C00C3EF9D52
:10449800FFEE9CFED082D083EEF0A3EFF0AF74EF76
:1044A8003395E0FEEF25E0FFEE33FE74222FF58210
:1044B80074003EF583E0FEA3E0FFC3EF9573E57259
:1044C8006480F8EE648098501FAF74EF3395E0FE77
:1044D800EF25E0FFEE33FE74222FF58274003EF5DF
:1044E80083E570F0A3E571F01250D974062574F5D0
:1044F80074900028E0FEA3E0FFEF4E705CE576B410
:104508000526301B230574AF74D3EF648094934061
:1045180003757400C21BAF74EF3395E0FE90003E44
:10452800EEF0A3EFF01250D9E5766403600302457C
:10453800B7301B7B1574AF74C3EF6480948050034D
:10454800757413C21BAF74EF3395E0FE90003EEE16
:10455800F0A3EFF01250D98056E576B40526301B4B
:10456800230574AF74D3EF6480949240037574008C
:10457800C21BAF74EF3395E0FE90003EEEF0A3EF60
:10458800F01250D9E576B40326301B231574AF74A6
:10459800C3EF648094805003757412C21BAF74EF2C
:1045A8003395E0FE90003EEEF0A3EFF01250D9E50F
:1045B80076B40102D21BE5765406FFEF6010900036
:1045C8003EE0FEA3E0FFEF64094E7002C20F9002C6
:1045D80005E0FEA3E0FF900028E0FCA3E0FDED6FFE
:1045E8007002EC6E6002C20F900028E0FEA3E0FFAC
:1045F800900205EEF0A3EFF030A302D21A20A30A2E
:0A460800301A07C21AA20FB3920F76
:014612002285
:104FD50012514474A012515C740212515C9000107D
:104FE5007C03E012511D12515CA3DCF6E012511D49
:104FF500F5F0A3A3E0030354C045F012515C900003
:1050050014E012511D12515CC2B4125137125144B1
:1050150074A012515C74F012515CA3E012515CC291
:10502500B41251372212514474A012515C74021209
:10503500515C12514474A00412515C90001012513D
:1050450081125125F0A3125194125181125125F06C
:10505500A3125194125181125125F0A312519412A9
:105065005181FB543F125125F0A3125194125181E5
:10507500FA541F125125F0EB23235403FD12518ED0
:10508500C2B412513712514474A012515C74F0121B
:10509500515C12514474A00412515C125181FB54AD
:1050A50003C39D2405838007030201000302012B2E
:1050B500A3F0F5F012518EC2B41251371251447457
:1050C500A012515C74F012515CE5F012515CC2B44F
:1050D500125137227AA07B807C1E9000221251D477
:1050E500227AA07B8012519CED900022F07AA0A339
:1050F5007C1D125209227AA07BD07C109000681288
:1051050051D4227AA07BD012519CED900068F07AA0
:01511500A0F9
:10511600A37C0F1252092275F00A84C425F022C01E
:10512600E0C4540F75F00AA4F5F0D0E0540F25F052
:105136002200D2B5000000D2B400000000221251B5
:1051460037C2B4000000C2B500000022D2B500008C
:1051560000C2B50000227E083392B4125152DEF826
:1051660033D2B40000A2B450040000A2B4125152CB
:10517600400122C2B40000125137227E08A2B43385
:1051860000125152DEF7C322D2B412515222C2B4D7
:10519600125152D2B422125144EA12515CEB12510E
:1051A6005C125144EA0412515C125181FD12518E77
:1051B600C2B412513722125144EA12515CEB125119
:1051C6005CE612515C08DCF9C2B412513722125166
:1051D60044EA12515CEB12515CE012515CA3DCF91B
:1051E600C2B412513722125144EA0412515C8003B0
:1051F600125194125181F608DCF612518EC2B41285
:10520600513722125144EA0412515C800312519420
:0C521600125181F0A3DCF612518EC2B4DC
:0452220012513722CC
:104CDB00202020202531642E2530326420253032CF
:104CEB0062753A25303262753A2530326275202072
:104CFB0020200020202020253032642E25316420F6
:104D0B0025303262753A25303262753A253032627F
:104D1B00752020202000253033642E25316420207F
:104D2B00253032642E25316420415A2F454C3120D9
:104D3B00202000253033642E25316420202530328D
:104D4B00642E25316420415A2F454C3220202000FF
:104D5B00253033642E2531642020253032642E25F6
:104D6B0031642052412F444543202020002530330D
:104D7B00642E2531645720253032642E2531644E44
:104D8B00204C4F2F4C4120202000253032627520C3
:104D9B0020202530326275202025303262753A256D
:104DAB00303262753A253032627520202020002582
:104DBB0030352E31662020253032642E253164208B
:104DCB0020202020202025303264202000202B257D
:104DDB003031642E2530316420202B253031642E68
:104DEB002530316420434F52202053545020002D46
:104DFB002D2D2D2D2D2D2D2D2D2D20202020202026
:104E0B005354502000253033642E25316420202547
:104E1B003032642E25316420414E542020253164DC
:104E2B002E2531642000202020204F2045203520C6
:104E3B004A2046204C20202020200020202020200B
:104E4B00202020454D452020202020202020200000
:104E5B0020416E74656E6E6120436F6E74726F6C61
:104E6B006C65722000202020202020207620372EF9
:104E7B00322020202020202020002020204A414EBC
:104E8B004645424D41524150524D41594A554E4A69
:104E9B00554C4155475345504F43544E4F5644453F
:104EAB0043004D4F4F4E202053554E202020434161
:104EBB005353494F4359474E555353414749545404
:104ECB005441555255534C454F202020415155418B
:104EDB00522E52412F444543415A2F454C32415A91
:104EEB002F454C3100326D3A37303A32333A313349
:104EFB003A39636D36636D31304732344700205396
:104F0B0053492031306269742837323029202020F0
:104F1B0020202053534931316269742831383030A5
:104F2B0029202020202020535349313262697428D4
:104F3B0033363030292020202020205353495F67FF
:104F4B0072617928343039362920202020202041E5
:104F5B00322D532D532031322062697420202020B2
:104F6B0020204D414232355F31306269743130322D
:104F7B003420202020204D414232355F313162698F
:104F8B00743230343820202020204D414232355F9E
:104F9B0031326269743430393620202020204D4163
:104FAB004232385F31326269743430393620202016
:104FBB002020000F0C09010306171D664C03090383
:0A4FCB00090309030956010102045D
:10002E00E57664016003125D10201403020663C2BC
:10003E001430190C900028E0FEA3E0FFEF4E601183
:10004E0090003EE0FEA3E0FFEF64134E600302015A
:10005E00FB90003CE0FEA3E0FFC3EF9404EE64804F
:10006E0094804003020108AF1CAE1B126E6DEF248C
:10007E0005FFEE3400FE7C007D0A121EDC9000E0CF
:10008E00EEF0A3EFF07B017A007980C003C002C0CE
:10009E00017BFF7A4C79DB9000F3EBF0A3EAF0A33F
:1000AE00E9F09000E0E0FEA3E0FF7C007D64121E0C
:1000BE00DC9000F6EEF0A3EFF09000E0E0FEA3E09F
:1000CE00FF7C007D64121EDC9000F8ECF0A3EDF0D6
:1000DE00900012E0FF9000FAEFF0900011E0FF9018
:1000EE0000FBEFF0900010E0FF9000FCEFF0D0016D
:1000FE00D002D003123DAA020198AF1CAE1B126EA5
:10010E006DEF2405FFEE3400FE7C007D0A121EDC2E
:10011E009000E0EEF0A3EFF07B017A007980C0034F
:10012E00C002C0017BFF7A4C79FE9000F3EBF0A386
:10013E00EAF0A3E9F09000E0E0FEA3E0FF7C007D92
:10014E000A121EDC9000F6EEF0A3EFF09000E0E055
:10015E00FEA3E0FF7C007D0A121EDC9000F8ECF09E
:10016E00A3EDF0900012E0FF9000FAEFF090001176
:10017E00E0FF9000FBEFF0900010E0FF9000FCEF2E
:10018E00F0D001D002D003123DAA751500D3E515AB
:10019E00648094825042AF1590003DE0FE75F003EE
:1001AE00EEA4F58285F083E5822FF582E43583F5A2
:1001BE0083E58224F0F582E583344EF583E493FFE4
:1001CE00AE15EEFD3395E0FC74802DF58274003C87
:1001DE00F583EFF0051580B5C3E51B648094804070
:1001EE00030205F3900083742DF00205F390003E98
:1001FE00E0FEA3E0FFEF640A4E601190003EE0FEC9
:10020E00A3E0FFEF640B4E600302029F7B017A00B6
:10021E007980C003C002C0017BFF7A4D7921900026
:10022E00F3EBF0A3EAF0A3E9F090002AE0FEA3E0DE
:10023E00FF7C007D0A121EDC9000F6EEF0A3EFF0BC
:10024E0090002AE0FEA3E0FF7C007D0A121EDC90E7
:10025E0000F8ECF0A3EDF090002CE0FEA3E0FF7CA4
:10026E00007D0A121EDC9000FAEEF0A3EFF0900073
:10027E002CE0FEA3E0FF7C007D0A121EDC9000FC49
:10028E00ECF0A3EDF0D001D002D003123DAA02058E
:10029E00F390003EE0FEA3E0FFEF640C4E60119081
:1002AE00003EE0FEA3E0FFEF640D4E600302034349
:1002BE007B017A007980C003C002C0017BFF7A4DBA
:1002CE00793E9000F3EBF0A3EAF0A3E9F090002E54
:1002DE00E0FEA3E0FF7C007D0A121EDC9000F6EE2D
:1002EE00F0A3EFF090002EE0FEA3E0FF7C007D0A6D
:1002FE00121EDC9000F8ECF0A3EDF0900030E0FE62
:10030E00A3E0FF7C007D0A121EDC9000FAEEF0A343
:10031E00EFF0900030E0FEA3E0FF7C007D0A121E9D
:10032E00DC9000FCECF0A3EDF0D001D002D0031273
:10033E003DAA0205F390003EE0FEA3E0FFEF640E3F
:10034E004E601190003EE0FEA3E0FFEF640F4E60A2
:10035E0003020426900034E0FEA3E0FFEF247CFFAE
:10036E00EE34FCFE90007CEEF0A3EFF090007CE00B
:10037E00FEA3E0FF126E6D7C007D0A121EDCC0062D
:10038E00C00790007CE0FEA3E0FF126E6D7C007D46
:10039E000A121EDC9000FCECF0A3EDF0D007D006A4
:1003AE009000FAEEF0A3EFF07B017A007980C003A3
:1003BE00C002C0017BFF7A4D795B9000F3EBF0A396
:1003CE00EAF0A3E9F0900032E0FEA3E0FF7C007DAE
:1003DE000A121EDC9000F6EEF0A3EFF0900032E071
:1003EE00FEA3E0FF7C007D0A121EDC9000F8ECF00C
:1003FE00A3EDF0D001D002D003123DAA90007CE014
:10040E00FEA3E0FFC3EE6480948040030205F390E8
:10041E000086742DF00205F390003EE0FEA3E0FF8F
:10042E00EF64104E601190003EE0FEA3E0FFEF641B
:10043E00114E600302054D900036E0FEA3E0FFEF83
:10044E0024F8FFEE34F8FE90007EEEF0A3EFF0906D
:10045E000038E0FEA3E0FFEF247CFFEE34FCFE90BC
:10046E00007CEEF0A3EFF090007EE0FEA3E0FF1222
:10047E006E6D7C007D0A121EDCC006C00790007EE9
:10048E00E0FEA3E0FF126E6D7C007D0A121EDCC042
:10049E0004C00590007CE0FEA3E0FF126E6D7C00B0
:1004AE007D0A121EDCC006C00790007CE0FEA3E0B1
:1004BE00FF126E6D7C007D0A121EDC9000FCECF0CB
:1004CE00A3EDF0D007D0069000FAEEF0A3EFF0D037
:1004DE0005D0049000F8ECF0A3EDF0D007D0069014
:1004EE0000F6EEF0A3EFF07B017A007980C003C036
:1004FE0002C0017BFF7A4D79789000F3EBF0A3EA0E
:10050E00F0A3E9F0D001D002D003123DAA90007EF4
:10051E00E0FEA3E0FFC3EE64809480500690008559
:10052E007445F090007CE0FEA3E0FFC3EE6480947F
:10053E008040030205F390008B7453F00205F37BA9
:10054E00017A007980C003C002C0017BFF7A4D7929
:10055E00959000F3EBF0A3EAF0A3E9F0900013E01E
:10056E00FF9000F6EFF0900015E0FF9000F7EFF02F
:10057E00900012E0FF9000F8EFF0900011E0FF9075
:10058E0000F9EFF0900010E0FF9000FAEFF0D001CC
:10059E00D002D003123DAA751500D3E515648094E0
:1005AE00825042AF15900014E0FE75F003EEA4F5F4
:1005BE008285F083E5822FF582E43583F583E5822B
:1005CE002485F582E583344EF583E493FFAE15EE74
:1005DE00FD3395E0FC74822DF58274003CF583EFBB
:1005EE00F0051580B5900028E0FEA3E0FFC3EF9460
:1005FE0002EE64809480503290003EE0FEA3E0FF55
:10060E00C3EF940AEE64809480401390003EE0FEA7
:10061E00A3E0FFD3EF9411EE64809480400C900021
:10062E00927444F09000937445F07F00125D227531
:10063E001500D3E51564809493501AAF15EF3395DA
:10064E00E0FE74802FF58274003EF583E0FF125CAD
:10065E00E9051580DD201503020879C21590003ECC
:10066E00E0FEA3E0FFC3EF940AEE64809480401591
:10067E0090003EE0FEA3E0FFD3EF9411EE64809471
:10068E00805002C2199001E2E0F8A3E0F9A3E0FA6B
:10069E00A3E0FB900004E0FCA3E0FDA3E0FEA3E0DA
:1006AE00FF121A77126ED47B007A007920784112ED
:1006BE00196E7B007A007900783F12187D121BD0DC
:1006CE0090007CEEF0A3EFF09001E2E0F8A3E0F9E9
:1006DE00A3E0FAA3E0FB900078E0FCA3E0FDA3E02A
:1006EE00FEA3E0FF121A77126ED47B007A00790017
:1006FE00783F12187D121BD09000E2EEF0A3EFF0BF
:10070E007B017A007998C003C002C0017BFF7A4D4D
:10071E0079BA9000F3EBF0A3EAF0A3E9F09001E2CE
:10072E00E0F8A3E0F9A3E0FAA3E0FB90000CE0FCF4
:10073E00A3E0FDA3E0FEA3E0FF121A779000F612ED
:10074E00202890007CE0FEA3E0FF7C007D0A121EB4
:10075E00DC9000FAEEF0A3EFF090007CE0FEA3E058
:10076E00FF7C007D0A121EDC9000FCECF0A3EDF085
:10077E009000E2E0FEA3E0FF9000FEEEF0A3EFF0AB
:10078E00D001D002D003123DAA7F007E007D007CF6
:10079E0000900004E0F8A3E0F9A3E0FAA3E0FB1256
:1007AE001B14500690009E742DF0751500D3E515A0
:1007BE00648094855042AF15900029E0FE75F006D6
:1007CE00EEA4F58285F083E5822FF582E43583F57C
:1007DE0083E58224ADF582E583344EF583E493FF01
:1007EE00AE15EEFD3395E0FC74A42DF58274003C3D
:1007FE00F583EFF0051580B5900028E0FEA3E0FF2D
:10080E00C3EF9402EE64809480400E9000AA742090
:10081E00F09000AB7420F080217F007E007D007C84
:10082E0000900078E0F8A3E0F9A3E0FAA3E0FB1251
:10083E001B1450069000A9742DF0E5766401602B10
:10084E007F40125D22751500D3E515648094935098
:10085E001AAF15EF3395E0FE74982FF58274003EB3
:10086E00F583E0FF125CE9051580DD201603020911
:10087E00CAC216900022E0FEA3E0FFEF249CFFEE1A
:10088E0034FFFE126E6D90007EEEF0A3EFF090003E
:10089E0024E0FEA3E0FFEF249CFFEE34FFFE126E79
:1008AE006D90007CEEF0A3EFF03010030209417B57
:1008BE00017A0079B0C003C002C0017BFF7A4D7986
:1008CE00D89000F3EBF0A3EAF0A3E9F090007EE0FD
:1008DE00FEA3E0FF7C007D0A121EDC9000F6EEF017
:1008EE00A3EFF090007EE0FEA3E0FF7C007D0A12F5
:1008FE001EDC9000F8ECF0A3EDF090007CE0FEA37F
:10090E00E0FF7C007D0A121EDC9000FAEEF0A3EFF1
:10091E00F090007CE0FEA3E0FF7C007D0A121EDC5E
:10092E009000FCECF0A3EDF0D001D002D003123D0C
:10093E00AA80267B017A0079B0C003C002C0017B79
:10094E00FF7A4D79FA9000F3EBF0A3EAF0A3E9F009
:10095E00D001D002D003123DAA900022E0FEA3E007
:10096E00FFC3EF9464EE6480948050069000B174DF
:10097E002DF0900024E0FEA3E0FFC3EF9464EE643C
:10098E0080948050069000B7742DF0E57664016077
:10099E002B7F14125D22751500D3E5156480949398
:1009AE00501AAF15EF3395E0FE74B02FF582740038
:1009BE003EF583E0FF125CE9051580DD201703028A
:1009CE000BE3C217900027E0FFEF904FD293FFEF9B
:1009DE003395E0FEAC66AD67121ECA8E4A8F4B9001
:1009EE0001F9E0FEA3E0FF126E6D7C007D0A121E7F
:1009FE00DCC006C0079001F9E0FEA3E0FF126E6DA9
:100A0E007C007D0A121EDC9000FCECF0A3EDF0D011
:100A1E0007D0069000FAEEF0A3EFF07B017A007992
:100A2E00C8C003C002C0017BFF7A4E79109000F35C
:100A3E00EBF0A3EAF0A3E9F09001FBE0FEA3E0FFE8
:100A4E007C007D0A121EDC9000F6EEF0A3EFF09013
:100A5E0001FBE0FEA3E0FF7C007D0A121EDC90008D
:100A6E00F8ECF0A3EDF0AE4AAF4B7C007D0A121EFF
:100A7E00DC9000FEEEF0A3EFF0AE4AAF4B7C007DB3
:100A8E000A121EDC900100ECF0A3EDF0D001D002B2
:100A9E00D003123DAA9001F9E0FEA3E0FFC3EE647D
:100AAE0080948050069000CE742DF0A21CB3921C40
:100ABE00E508540CFFEFB40808201C059000D8E49C
:100ACE00F0E508540CFFEFB40409201C069000D882
:100ADE007401F0E508540CFFEFB40C09300F0690CA
:100AEE0000D8742AF0E5085403FFEFB40209301C55
:100AFE00069000D77402F0E5085403FFEFB4010925
:100B0E00301C069000D77403F0E5085403FFEFB4D1
:100B1E000309300F069000D7742AF090003EE0FED5
:100B2E00A3E0FFEF64124E6003020BB8751500D3FD
:100B3E00E515648094935042AF1590003BE0FE752E
:100B4E00F014EEA4F58285F083E5822FF582E4356C
:100B5E0083F583E5822409F582E583344FF583E43A
:100B6E0093FFAE15EEFD3395E0FC74C82DF582743F
:100B7E00003CF583EFF0051580B5AE4AAF4B7C0017
:100B8E007D0A121EDCEF2430FF9000D9EFF09000AA
:100B9E00DA742EF0AE4AAF4B7C007D0A121EDCAF2B
:100BAE0005EF2430FF9000DBEFF07F54125D2275CD
:100BBE001500D3E51564809493501AAF15EF339555
:100BCE00E0FE74C82FF58274003EF583E0FF125CE0
:100BDE00E9051580DDE576B4011490003FE0FFEFE6
:100BEE00904FBE93FF125D22125D07125D193018F1
:100BFE0003020D467B017A007980C003C002C0015A
:100C0E007BFF7A4E79319000F3EBF0A3EAF0A3E983
:100C1E00F0D001D002D003123DAA7B017A00799860
:100C2E00C003C002C0017BFF7A4E79469000F3EB01
:100C3E00F0A3EAF0A3E9F0D001D002D003123DAA4E
:100C4E007B017A0079B0C003C002C0017BFF7A4EEF
:100C5E00795B9000F3EBF0A3EAF0A3E9F0D001D0BA
:100C6E0002D003123DAA7B017A0079C8C003C002EC
:100C7E00C0017BFF7A4E79709000F3EBF0A3EAF09F
:100C8E00A3E9F0D001D002D003123DAA7F00125D7D
:100C9E0022751500D3E51564809493501AAF15EFA5
:100CAE003395E0FE74802FF58274003EF583E0FFED
:100CBE00125CE9051580DD7F40125D22751500D3AB
:100CCE00E51564809493501AAF15EF3395E0FE74DA
:100CDE00982FF58274003EF583E0FF125CE905154E
:100CEE0080DD7F14125D22751500D3E515648094A6
:100CFE0093501AAF15EF3395E0FE74B02FF5827452
:100D0E00003EF583E0FF125CE9051580DD7F54128D
:100D1E005D22751500D3E51564809493501AAF15B6
:100D2E00EF3395E0FE74C82FF58274003EF583E034
:090D3E00FF125CE9051580DD22BD
:106D3A00015100014F00015000014900C10FC10C6F
:0A6D4A00C10BC10EC110C10DC11133
:106E7F00752400D3E524648094A75004052480F37F
:016E8F0022E0
:106E9000752500D3E525648094935004052580F37F
:016EA00022CF
:106EA100752600D3E5266480949E5004052680F360
:016EB10022BE
:106EB200752700D3E5276480949E5004052780F34C
:016EC20022AD
:106EC300752800D3E5286480949E5004052880F338
:016ED300229C
:10609F00C290126E7F752E1F752D00E52DD39407BC
:1060AF005011E52EC313F52EA2D79290126E7F05D5
:1060BF002D80E8D290126E7FD292752903752AE84F
:1060CF00752E00309110E52A152A7002152914FF3C
:1060DF00AE29EF4E70ED126E90752D00E52DD39415
:1060EF00075013126E7FE52EC313F52E3091034325
:1060FF002E80052D80E6126E7FAF2E7E00EF752C61
:10610F0000F52B752903752AE8752E00309110E5DF
:10611F002A152A7002152914FFAE29EF4E70ED12C1
:10612F006E90752D00E52DD394075013126E7FE5F9
:10613F002EC313F52E309103432E80052D80E612CA
:10614F006E7FAF2E7E00EF252CF52CEE352BF52B29
:10615F00C3E52B648094805006752B00752C00D3FB
:10616F00E52C940FE52B6480948E4006752B0E75ED
:10617F002C0FC29220B20DC3740F952CF52C740EF8
:08618F00952BF52BAE2BAF2C74
:0161970022E5
:10637600C294126E7F75341F753300E533D39407CC
:106386005011E534C313F534A2D79294126E7F05EB
:106396003380E8D294126E7FD296752F037530E85B
:1063A600753400309510E53015307002152F14FF46
:1063B600AE2FEF4E70ED126E90753300E533D39429
:1063C600075013126E7FE534C313F534309503433B
:1063D6003480053380E6126E7FAF347E00EF75326F
:1063E60000F531752F037530E8753400309510E5EA
:1063F6003015307002152F14FFAE2FEF4E70ED12D0
:106406006E90753300E533D394075013126E7FE513
:1064160034C313F534309503433480053380E612D4
:106426006E7FAF347E00EF2532F532EE3531F53131
:10643600C3E531648094805006753100753200D30F
:10644600E532940FE5316480948E400675310E7501
:08645600320FC296AE31AF32E5
:01645E00221B
:10000E0012609F8E4D8F4E1263768E478F487566A7
:05001E000075670122DE
:10688A00D290D294D291D295756C00756D007568CC
:10689A0000756900753500D3E535648094895049DF
:1068AA00126EA1C290C294126EA1C3E5356480949F
:1068BA00895004D290D294E56D256DF56DE56C355D
:1068CA006CF56CE5692569F569E5683568F5682050
:1068DA009108056DE56D7002056C2095080569E55E
:1068EA006970020568053580AEC290C2947566006B
:1068FA00756705AE6CAF6D7C007D05121ECA8E4DA4
:10690A008F4E20B20DC3740B954EF54E740E954DF5
:10691A00F54DAE68AF697C007D05121ECA8E478FA1
:01692A004824
:01692B002249
:106A6600D290D294D291D295756C00756D007568EE
:106A760000756900753600D3E5366480948A5049FE
:106A8600126EA1C290C294126EA1C3E536648094C0
:106A96008A5004D290D294E56D256DF56DE56C357E
:106AA6006CF56CE5692569F569E5683568F5682072
:106AB6009108056DE56D7002056C2095080569E580
:106AC6006970020568053680AEC290C2947566008C
:106AD600756702E56D25E0F54EE56C33F54D20B2A0
:106AE6000DC3740E954EF54E740E954DF54DE56934
:096AF60025E0F548E56833F54799
:016AFF002274
:106C2600D290D294D291D295756C00756D0075682C
:106C360000756900753700D3E5376480948B504939
:106C4600126EA1C290C294126EA1C3E537648094FD
:106C56008B5004D290D294E56D256DF56DE56C35BB
:106C66006CF56CE5692569F569E5683568F56820B0
:106C76009108056DE56D7002056C2095080569E5BE
:106C86006970020568053780AEC290C294756600C9
:106C9600756701856C4D856D4E20B20DC3740F95D9
:0F6CA6004EF54E740E954DF54D8568478569483E
:016CB50022BC
:105D6700D292D291756C00756D00126EB2753800C3
:105D7700D3E5386480948F5025D290126EB2C290CA
:105D8700126EB2E56D256DF56DE56C356CF56C2021
:105D97009108056DE56D7002056C053880D2C290DB
:105DA700C292E56DAE6C7806CEC313CE13D8F9F563
:105DB7006D8E6CAC6CAD6DE4121B977B007A00792D
:105DC70034784412196E7B007A0079807844121A6D
:105DD70077121BD07C007D05121ECA8E4D8F4E2078
:105DE700B20DC3740B954EF54E740E954DF54D12CD
:105DF7006EB2756600756705D296D295756800759F
:105E07006900126EB2753800D3E5386480948F50FC
:105E170025D294126EB2C294126EB2E5692569F565
:105E270069E5683568F5682095080569E5697002D0
:105E37000568053880D2C294C296E569AE687806CF
:105E4700CEC313CE13D8F9F5698E68AC68AD69E493
:105E5700121B977B007A007934784412196E7B0005
:105E67007A0079807844121A77121BD07C007D055E
:075E7700121ECA8E478F487E
:015E7E002201
:105E7F00D292D291756C00756D00126EB2753900A9
:105E8F00D3E5396480948F5025D290126EB2C290B0
:105E9F00126EB2E56D256DF56DE56C356CF56C2008
:105EAF009108056DE56D7002056C053980D2C290C1
:105EBF00C292E56DAE6C7805CEC313CE13D8F9F54B
:105ECF006D8E6CAC6CAD6DE4121B977B007A007914
:105EDF00E1784412196E7B007A0079007845121A26
:105EEF0077121BD0EF25E0F54EEE33F54D20B20DB6
:105EFF00C3740E954EF54E740E954DF54D126EB250
:105F0F00756600756702D296D2957568007569003F
:105F1F00126EB2753900D3E5396480948F5025D253
:105F2F0094126EB2C294126EB2E5692569F569E5F5
:105F3F00683568F5682095080569E5697002056898
:105F4F00053980D2C294C296E569AE687805CEC392
:105F5F0013CE13D8F9F5698E68AC68AD69E4121BDE
:105F6F00977B007A0079E1784412196E7B007A00F2
:105F7F0079007845121A77121BD0EF25E0F548EE1D
:035F8F0033F547A0
:015F920022EC
:105F9300D292D291756C00756D00126EB2753A0093
:105FA300D3E53A6480948F5025D290126EB2C2909A
:105FB300126EB2E56D256DF56DE56C356CF56C20F3
:105FC3009108056DE56D7002056C053A80D2C290AB
:105FD300C292E56CC4F854F0C868F56CE56DC4541E
:105FE3000F48F56DAC6CAD6DE4121B977B007A0026
:105FF3007961784512196E7B007A007980784512B1
:106003001A77121BD08E4D8F4E20B20DC3740F958D
:106013004EF54E740E954DF54D126EB275660075C4
:106023006701D296D295756800756900126EB275D4
:106033003A00D3E53A6480948F5025D294126EB21D
:10604300C294126EB2E5692569F569E5683568F5AC
:10605300682095080569E56970020568053A80D2EC
:10606300C294C296E568C4F854F0C868F568E56957
:10607300C4540F48F569AC68AD69E4121B977B0003
:106083007A007961784512196E7B007A00798078FD
:0B60930045121A77121BD08E478F4871
:01609E0022DF
:1057FC00D292D291756C00756D00126EC3753B0020
:10580C00D3E53B6480948F5025D290126EC3C29026
:10581C00126EC3E56D256DF56DE56C356CF56C2080
:10582C009108056DE56D7002056C053B80D2C29048
:10583C00C292E56CC4F854F0C868F56CE56DC454BC
:10584C000F48F56DD3E56D9559E56C955840188565
:10585C006C62856D63856C58856D59E56D24FFF51B
:10586C0057E56C34FFF556C3E56D9557E56C9556C9
:10587C00501EE56D2401F563E56C3400F562856C12
:10588C0056856D57E56D2401F559E56C3400F558D6
:10589C00AC62AD63EC121B977B007A0079617845A2
:1058AC0012196E7B007A0079807845121A77121BD8
:1058BC00D08E4D8F4E20B20DC3740F954EF54E7495
:1058CC000E954DF54D126EB2756600756701D29648
:1058DC00D295756800756900126EC3753B00D3E5EF
:1058EC003B6480948F5025D294126EC3C294126E76
:1058FC00C3E5692569F569E5683568F5682095089B
:10590C000569E56970020568053B80D2C294C296B0
:10591C00E568C4F854F0C868F568E569C4540F48E4
:10592C00F569D3E5699555E5689554401885685E29
:10593C0085695F856854856955E56924FFF553E5EC
:10594C006834FFF552C3E5699553E5689552501ECE
:10595C00E5692401F55FE5683400F55E85685285DC
:10596C006953E5692401F555E5683400F554AC5EDE
:10597C00AD5FEC121B977B007A00796178451219A8
:10598C006E7B007A0079807845121A77121BD08EC4
:03599C00478F48EA
:01599F0022E5
:10628800D290D294D291D295756C00756D007568D4
:1062980000756900753C00D3E53C6480948B5053CD
:1062A800C290C294753D00D3E53D64809482500449
:1062B800053D80F3C3E53C6480948B5004D290D2B2
:1062C80094E56D256DF56DE56C356CF56CE5692526
:1062D80069F569E5683568F568209108056DE56D2B
:1062E8007002056C2095080569E569700205680566
:1062F8003C80A4C290C294756600756701AF6DAE0C
:106308006C126E558E6C8F6DAF69AE68126E558EBD
:10631800688F69AC6CAD6DE4121B977B007A0079CD
:1063280061784512196E7B007A0079807845121AD7
:1063380077121BD08E4D8F4E20B20DC3740F954E21
:10634800F54E740E954DF54DAC68AD69E4121B978A
:106358007B007A007961784512196E7B007A0079A2
:0D636800807845121A77121BD08E478F489F
:016375002205
:10384D00E54C64326003300D61C3E56F954EF56153
:10385D00E56E954DF560C374089548FF740795475F
:10386D00FE126E6DC374849FFF74039EFEC3E56BE1
:10387D009FF55BE56A9EF55AC3E5489408E54764F4
:10388D00809487400BC3E4955BF55BE4955AF55A3C
:10389D00C210C20E900068E560F0A3E561F09000E3
:1038AD006AE55AF0A3E55BF0C20D20101B20B303AF
:1038BD00300E03301112D210D20E90006CE4F0A332
:1038CD007401F01250FBC21130101D20B303300EE5
:1038DD0003301114C210D20E1250E690006CE4F0B9
:1038ED00A3E4F01250FBC21120B304054C80057502
:1038FD004C00C20E301074E561254EF54EE5603575
:10390D004DF54DD3E54E940FE54D6480948E400CEE
:10391D0074F0254EF54E74F1354DF54DC3E54D64FE
:10392D00809480500C7410254EF54E740E354DF567
:10393D004DE55B2548F548E55A3547F547D3E5484C
:10394D00940FE5476480948E400C74F02548F5483B
:10395D0074F13547F547C3E54764809480500C7486
:10396D00102548F548740E3547F547C3740895483A
:10397D00FF74079547FE126E6DC374849FF54874EE
:10398D00039EF5479001FBE54DF0A3E54EF0900148
:10399D00F9E547F0A3E548F0E56F24F8F55DE56E30
:1039AD0034F8F55CE54E24F8F565E54D34F8F5642D
:1039BD00C3E55C64809480500C7410255DF55D74D6
:1039CD000E355CF55CC3E56464809480500C741016
:1039DD002565F565740E3564F56430105A90003820
:1039ED00E0FEA3E0FFC3EF9484EE64809483400F68
:1039FD00C3E56F954EF53FE56E954DF53E800DC3D4
:103A0D00E55D9565F53FE55C9564F53ED3E56B9415
:103A1D0000E56A648094804010C3E56B9548F541DC
:103A2D00E56A9547F540023AECC3E49548F541E463
:103A3D009547F540023AEC900038E0FEA3E0FFC355
:103A4D00EF9484EE648094834025900022E0FEA3E1
:103A5D00E0FFE56F2FFFE56E3EFEEF249CFFEE3499
:103A6D00FFFEC3EF954EF53FEE954DF53E8023904D
:103A7D000022E0FEA3E0FFE55D2FFFE55C3EFEEFDB
:103A8D00249CFFEE34FFFEC3EF9565F53FEE956484
:103A9D00F53ED3E56B9400E56A64809480402590F3
:103AAD000024E0FEA3E0FFE56B2FFFE56A3EFEEF8D
:103ABD00249CFFEE34FFFEC3EF9548F541EE95478C
:103ACD00F540801B900024E0FEA3E0FFEF249CFF57
:103ADD00EE34FFFEC3EF9548F541EE9547F5407581
:103AED00080F200F03023D24AE4AAF4B7C007D0230
:103AFD00121EDCD3E53F9FEE6480F8E53E648098AE
:103B0D004024E54620E5067551007550000551AF7E
:103B1D0051EFD394504003755150E551C3940A4071
:103B2D005053080E804BAE4AAF4B7C007D02121EE7
:103B3D00DCC3E49FFFE49EFEC3E53F9FEE6480F887
:103B4D00E53E6480985024E54620E40675510075E5
:103B5D0050000551AF51EFD394504003755150E5CE
:103B6D0051C3940A400B53080D80067551007550D2
:103B7D0000AE4AAF4B7C007D02121EDCD3E5419FA7
:103B8D00EE6480F8E5406480984024E54620E70621
:103B9D00754F00754900054FAF4FEFD3945040035B
:103BAD00754F50E54FC3940A405D53080B8058AED6
:103BBD004AAF4B7C007D02121EDCC3E49FFFE49EE6
:103BCD00FEC3E5419FEE6480F8E540648098503176
:103BDD00D3E5489400E547648094804024E5462071
:103BED00E606754F00754900054FAF4FEFD3945062
:103BFD004003754F50E54FC3940A400B530807809F
:103C0D0006754F00754900AF3FAE3E126E6D8E4288
:103C1D008F43C374289543FFE49542FEEF7802C3AA
:103C2D0033CE33CED8F9FFAD507C00C3EF9DF545B3
:103C3D00EE9CF544C3E544648094805006754400C1
:103C4D00754500E551C39450501DAF517E007C0069
:103C5D007D7F121ECA7C007D50121EDCEF2480FF7A
:103C6D00EF64FFF5FA8027C3E5439428E5426480AD
:103C7D0094805017E550C394A050100550C3E544EF
:103C8D006480948040088545FA800375FA00AF4141
:103C9D00AE40126E6D8E428F43C374289543FFE480
:103CAD009542FEEF7802C333CE33CED8F9FFAD493E
:103CBD007C00C3EF9DF545EE9CF544C3E54464805F
:103CCD0094805006754400754500E54FC3945050DF
:103CDD001DAF4F7E007C007D7F121ECA7C007D5083
:103CED00121EDCEF2480FFEF64FFF5FE803BC3E581
:103CFD00439428E542648094805017E549C394A00D
:103D0D0050100549C3E54464809480401C8545FEF0
:103D1D00801775FE008012755100755000754F00AB
:103D2D0075490075FA0075FE00E508C454F0FFEF03
:073D3D00240FF5468546A0A6
:013D4400225C
:106DEE004310000043D8000044A2000045110000EB
:106DFE004554800045B400004622000046BD000008
:106E0E0000C700C70002000A0E0F03840E0F038492
:106E1E000001000100000000000000000000000062
:106D5400011400011663011200011700011A00C199
:036D640013C192C6
:0300030002652172
:10652100C0E0C083C08263A201C083C082C0D075B5
:10653100D000C006C00720124F20134CD2B330B395
:10654100020512051AAF1AC3EF64809488401CAF8C
:1065510017EF3395E0FE74402FF58274003EF5830A
:10656100E512F07512000517751A00E5122512F5EE
:1065710012C3E51764809484404F751700D21390BD
:106581000048E0FF8F12804120123E30133BE5129C
:106591002512F512A2D792B3051AAF1AC3EF648080
:1065A1009488401A0517AF17EF3395E0FE74482F12
:1065B100F58274003EF583E0FF8F12751A00C3E582
:1065C10017648094A04002D212D007D006D0D0D058
:0D65D10082D08363A201D082D083D0E0325B
:10544E00900048E56EF0A3E56FF0E56B2484FFE570
:10545E006A3403FE90004AEEF0A3EFF09001FBE0F9
:10546E00FEA3E0FF90004CEEF0A3EFF09001F9E008
:10547E00FEA3E0FFEF2484FFEE3403FE90004EEE19
:10548E00F0A3EFF0E50B2484FFE50A3403FE900051
:10549E0050EEF0A3EFF0900022E0FEA3E0FF9000AC
:1054AE0052EEF0A3EFF0900024E0FEA3E0FF900098
:1054BE0054EEF0A3EFF0900028E0FEA3E0FF900082
:1054CE0056EEF0A3EFF0900058E54AF0A3E54BF04E
:1054DE00300F0B90005AE4F0A37401F08008900096
:1054EE005AE4F0A3E4F0900015E0FFEF3395E0FEF0
:1054FE0090005CEEF0A3EFF0900014E0FFEF339518
:10550E00E0FE90005EEEF0A3EFF0900013E0FFEFF0
:10551E003395E0FE900060EEF0A3EFF0900012E005
:10552E00FFEF3395E0FE900062EEF0A3EFF09000F7
:10553E0011E0FFEF3395E0FE900064EEF0A3EFF084
:10554E00900041E0F516900040E4F0A37463F0C3C0
:10555E00E51664809488400302563FC3E5166480C6
:10556E009480500302563F900042E0F518A3E0F5F8
:10557E0019AF16EF3395E0FEEF25E0FFEE33FE7424
:10558E000E2FF582746E3EF583E493FE740193FF45
:10559E00D3E5199FEE6480F8E5186480984021AF3A
:1055AE0016EF3395E0FEEF25E0FFEE33FE740E2F7F
:1055BE00F582746E3EF583E493F518740193F51934
:1055CE00AF16EF3395E0FEEF25E0FFEE33FE741ECF
:1055DE002FF582746E3EF583E493FE740193FFC340
:1055EE00E5199FEE6480F8E5186480985021AF1697
:1055FE00EF3395E0FEEF25E0FFEE33FE741E2FF540
:10560E0082746E3EF583E493F518740193F519AF29
:10561E0016EF3395E0FEEF25E0FFEE33FE74222FFA
:10562E00F58274003EF583E518F0A3E519F01250EB
:0C563E00D9E516B40805A20FB3920F22A4
:03002B0002645F0D
:10645F00C0E0C0F0C083C08263A201C083C082C00D
:10646F00D075D000C000C001C002C003C004C00579
:10647F00C006C00775A61E75A6E11509AF09EF7016
:10648F006D75090453907790003AE0FEA3E0FFEF9B
:10649F008EF01220AB64CC000064D1000164D600F2
:1064AF000264DB000364E0000464E5000564EA00B5
:1064BF000664EF000764F40008000064F712688AAE
:1064CF008026126A668021126C26801C12628880D8
:1064DF001712000E8012125D67800D125E7F80080A
:1064EF00125F9380031257FC43908812384DC2CF2E
:1064FF00D007D006D005D004D003D002D001D000F1
:10650F00D0D0D082D08363A201D082D083D0F0D0FC
:02651F00E03268
:03002300026CB6B6
:106CB600C0E0C0F0C083C08263A201C083C082C0AE
:106CC600D075D000C000C001C002C003C004C0051A
:106CD600C006C007C2AC30981AC298E599B43F0303
:106CE600125226E599B4210B12564AD214D215D265
:106CF60016D217C299D2ACD007D006D005D004D090
:106D060003D002D001D000D0D0D082D08363A201BC
:096D1600D082D083D0F0D0E0322D
:03000B000265DEAD
:1065DE00C0E0C0F0C083C08263A201C083C082C08D
:1065EE00D075D000C000C001C002C003C004C005F9
:1065FE00C006C007758A00758C4C75A61E75A6E17F
:10660E000514AF14C3EF6480948A401630121375CC
:10661E001400751700751A00C213C21275120012FB
:10662E00544EE51375F007121E50AFF0EF701B12AB
:10663E0041C8301804D214D217E57660073018041A
:10664E00D215D21612002E12502A1513AF13EF7058
:10665E000C75134ED218301804D215D216D007D09E
:10666E0006D005D004D003D002D001D000D0D0D0B7
:0F667E0082D08363A201D082D083D0F0D0E032EB
:10224500758FFF758921758DFF438780759850D2ED
:102255008CD28ED2CA75CB4C75CA0043B71143B820
:1022650021D28875D90243D84075DA4275DE42C25B
:10227500187513467509017F02125CB1125CFE7573
:102285007700900040E4F0A37463F020A003126B84
:102295000075A8B275A7071250E6125108C20F9033
:1022A500006CE0FEA3E0FFEF4E6004D2108002C296
:1022B50010900068E0F560A3E0F56190006AE0F534
:1022C5005AA3E0F55BE57670FC900036E0FCA3E0F0
:1022D500FDEC121B977B007A0079207841121A7762
:1022E5007B007A00793478C312187D9001E2E0F81A
:1022F500A3E0F9A3E0FAA3E0FB12196E90001E1209
:102305002028900038E0FCA3E0FDEC121B977B0031
:102315007A0079207841121A777B007A0079B478AF
:10232500C212187D9001E2E0F8A3E0F9A3E0FAA358
:10233500E0FB12196E90001A122028900011E0FCA3
:10234500EC121B9C7B007A0079B47844121A77C092
:1023550004C005C006C007900012E0FCEC121B9CEF
:102365007B007A0079C07841121A77A804A905AADA
:1023750006AB07D007D006D005D00412187DC004DF
:10238500C005C006C007900010E0FCEC121B9C7B4A
:10239500007AC079A87847121A77A804A905AA0671
:1023A500AB07D007D006D005D00412187D900044A5
:1023B500122028900014E0FFEF3395E0FEFDFCEFBE
:1023C5002409FFEE3400FEED3400FDEC3400FC7B07
:1023D5000C7A0079007800126D68A804A905AA0690
:1023E500AB07900015E0FFEF3395E0FEFDFCEF2411
:1023F500D0FFEE3407FEED3400FDEC3400FCEB2F8E
:10240500FFEA3EFEE93DFDE83CFC7B077A007900EA
:102415007800121F287B047A0079007800126D6815
:10242500C004C005C006C007900015E0FFEF339556
:10243500E0FEFDFC7B6F7A0179007800121F28D041
:1024450003D002D001D000C3EF9BFFEE9AFEED99B9
:10245500FDEC98FCC004C005C006C007900014E060
:10246500FFEF3395E0FEFDFC7B137A0179007800E0
:10247500121F287B097A0079007800126D68A8047C
:10248500A905AA06AB07D007D006D005D004EB2FC7
:10249500FBEA3EFAE93DF9E83CF8900013E0FFEF6E
:1024A5003395E0FEFDFCEB2FFFEA3EFEE93DFDE83E
:1024B5003CFCEF247AF511EE34E0F510ED3400F52F
:1024C5000FEC3400F50E900028E0FEA3E0FFEF646A
:1024D500014E70487B017A007908C003C002C00133
:1024E5007B017A0079789001ABEBF0A3EAF0A3E9E0
:1024F500F0AF11AE10AD0FAC0E9001AE12202890CA
:102505000044E0FCA3E0FDA3E0FEA3E0FF9001B2E0
:10251500122028D001D002D003124613900028E0E3
:10252500FEA3E0FFEF4E600302275A7B017A007994
:1025350008C003C002C0017B017A007978900123AD
:10254500EBF0A3EAF0A3E9F0AF11AE10AD0FAC0EBE
:10255500900126122028900044E0FCA3E0FDA3E0B2
:10256500FEA3E0FF90012A122028D001D002D0035B
:10257500122B2F90001AE0FCA3E0FDA3E0FEA3E0E0
:10258500FF1259E87B547AE37945784012196EC0F9
:1025950004C005C006C007900016E0FCA3E0FDA33B
:1025A500E0FEA3E0FF1259FEA804A905AA06AB07A1
:1025B500D007D006D005D00412196EC004C005C0DE
:1025C50006C007900078E0FCA3E0FDA3E0FEA3E0D1
:1025D500FF1259E8A804A905AA06AB07D007D0063B
:1025E500D005D00412196EC004C005C006C007AFDF
:1025F50011AE10AD0FAC0EC004C005C006C0077FFC
:10260500AB7EAA7D2A7C3C900044E0F8A3E0F9A3C8
:10261500E0FAA3E0FB12187D90015E122028D00796
:10262500D006D005D004120D47C004C005C006C0B1
:1026350007AF11AE10AD0FAC0EC004C005C006C08B
:10264500077FAB7EAA7D2A7CBC900044E0F8A3E01E
:10265500F9A3E0FAA3E0FB12187D90015E12202891
:10266500D007D006D005D004120D47D003D002D034
:1026750001D0001218797B007A0079877843121A05
:1026850077A804A905AA06AB07D007D006D005D0C0
:102695000412187D7B007A00797A784412196E123B
:1026A5001BD08E0C8F0D90003CE0FEA3E0FFC3EF26
:1026B5009404EE64809480504FAC0CAD0DEC121B6D
:1026C50097C004C005C006C00790003CE0FEA3E02B
:1026D500FFEF7802C333CE33CED8F9FF74EE2FF572
:1026E50082746D3EF583121FF8D007D006D005D051
:1026F5000412196E7B007A00797A7844121A7712DF
:102705001BD08E1B8F1C804DAC0CAD0DEC121B9796
:10271500C004C005C006C00790003CE0FEA3E0FF72
:10272500EF7802C333CE33CED8F9FF74EE2FF5829E
:10273500746D3EF583121FF8D007D006D005D0047E
:1027450012196E7B007A40791C7846121A77121B93
:10275500D08E1B8F1C900028E0FEA3E0FFEF6402E3
:102765004E70149000781220343F82D0E590000816
:1027750012203440C39DB2900028E0FEA3E0FFEF95
:1027850064034E70149000781220343F3566CF9064
:10279500000812203440A73B64900028E0FEA3E027
:1027A500FFEF64044E7014900078122034BF018F3F
:1027B500C590000812203440953F7D900028E0FE2A
:1027C500A3E0FFEF64054E70149000781220343EAC
:1027D500C44D019000081220343FB9168790002897
:1027E500E0FEA3E0FFEF64064E701490007812201F
:1027F500343F32B6AE900008122034401F2B0290B1
:102805000028E0FEA3E0FFEF64074E701490007807
:102815001220340000000090000812203440BC7AD9
:10282500E1900028E0FEA3E0FFEF64084E7067909A
:102835000032E0FCA3E0FDEC121B977B007A0079E7
:10284500207841121A779001E2E0F8A3E0F9A3E0BD
:10285500FAA3E0FB12196E900008122028900034AC
:10286500E0FCA3E0FDEC121B977B007A0079207851
:1028750041121A777B007A0079B478C212187D90DC
:1028850001E2E0F8A3E0F9A3E0FAA3E0FB12196E78
:10289500900078122028900028E0FEA3E0FFC3EF07
:1028A5009409EE6480948040030229AE900044E0D0
:1028B500FCA3E0FDA3E0FEA3E0FFC004C005C00645
:1028C500C007AF11AE10AD0FAC0E9001CE1220288F
:1028D500D007D006D005D0041249DB90018812201C
:1028E500287B017A00790CC003C002C0017B017A04
:1028F500007900900185EBF0A3EAF0A3E9F09000E0
:1029050008E0FCA3E0FDA3E0FEA3E0FF90018C122C
:102915002028900078E0FCA3E0FDA3E0FEA3E0FF03
:10292500900190122028D001D002D00312333690A6
:102935000028E0FEA3E0FFEF4E705A900000E0FC97
:10294500A3E0FDA3E0FEA3E0FF1259E87B007A5067
:1029550079C7784512196EC004C005C006C0079036
:1029650000E812203448B98C00D007D006D005D035
:10297500041269C9A804A905AA06AB07900000E0DE
:10298500FCA3E0FDA3E0FEA3E0FF1218799000048C
:102995001220288014900000E0FCA3E0FDA3E0FED7
:1029A500A3E0FF900004122028900028E0FEA3E099
:1029B500FFEF64094E705C90002EE0FCA3E0FDEC97
:1029C500121B977B007A0079207841121A779001C3
:1029D500E2E0F8A3E0F9A3E0FAA3E0FB12196E9098
:1029E500000C122028900030E0FCA3E0FDEC121B47
:1029F500977B007A0079207841121A779001E2E0FE
:102A0500F8A3E0F9A3E0FAA3E0FB12196E90000425
:102A1500122028900028E0FEA3E0FFEF640A4E7024
:102A25005C90002AE0FCA3E0FDEC121B977B007A8A
:102A35000079207841121A779001E2E0F8A3E0F9D5
:102A4500A3E0FAA3E0FB12196E90000C1220289067
:102A5500002CE0FCA3E0FDEC121B977B007A0079CB
:102A6500207841121A779001E2E0F8A3E0F9A3E09B
:102A7500FAA3E0FB12196E9000041220289001E2DF
:102A8500E0F8A3E0F9A3E0FAA3E0FB90000CE0FC7A
:102A9500A3E0FDA3E0FEA3E0FF121A777BCD7ACC7D
:102AA500794C783D12187D7B007A007920784112A7
:102AB500196E121BD08E6E8F6F9001E2E0F8A3E0C5
:102AC500F9A3E0FAA3E0FB900004E0FCA3E0FDA37A
:102AD500E0FEA3E0FF121A777BCD7ACC794C783DE6
:102AE50012187D7B007A007920784112196E121B2D
:102AF500D08E6A8F6B7F007E007D207C41900078B0
:102B0500E0F8A3E0F9A3E0FAA3E0FB12196E900147
:102B1500E2E0F8A3E0F9A3E0FAA3E0FB121A7712CA
:0A2B25001BD08E0A8F0B0222CA2279
:105C4A00EFC0E0C283740F125C7F7430125C8974F7
:105C5A0005125C7F7430125C897401125C7F7430A7
:105C6A00125C897401125C7FD0E0146002740844EB
:105C7A0020125C97227D000000DDFCD5E0F722545B
:105C8A00F053800F4280C282D283C28322C28280B2
:105C9A0002D282C0E0125CA5D0E0C454F053800F57
:105CAA004280D283C28322125C4A125CE3740612D7
:105CBA005C97125CE3740E125C97125CE374011237
:105CCA005C97125CE37440125C97125D30125CE3DD
:105CDA007480125C97125D1022740A125C7F22EFA4
:105CEA00C0E0125CE3D0E0125C9B22125CE3740217
:105CFA00125C9722125CE37401125C9722125CE335
:105D0A00740E125C9722125CE3740C125C972212D6
:105D1A005CE3740F125C9722EFC0E0125CE3D0E000
:105D2A004480125C9722905D3F7E28E493FF125CC8
:105D3A00E9A3DEF7220004040E0E1F1F00001F1F36
:105D4A000E0E04040000101C1F1C100000000107A6
:0D5D5A001F070100000E11171917110E0090
:106E55007A107B00EE6BFB8BF053F080ABF033EFD9
:086E650033FFEE33FEDAEE22EA
:106B9500900207EEF0A3EFF0900207E0FEA3E0FFFE
:106BA5007C037DE8121EDCEF2430F5993099FDC297
:106BB50099900207E0FEA3E0FF7C037DE8121EDC4E
:106BC5007E007F64CFCDCFCECCCE121EDCEF24303D
:106BD500F5993099FDC299900207E0FEA3E0FF7C8C
:106BE500007D64121EDC7E007F0ACFCDCFCECCCED9
:106BF500121EDCEF2430F5993099FDC299900207F9
:106C0500E0FEA3E0FF7C007D0A121EDCAF05EF2449
:106C150030F5993099FDC2997599003099FDC29961
:016C2500224C
:105226009001FD122034000186A020983E9001FDD9
:10523600E0FCA3E0FDA3E0FEA3E0FFEC4D4E4F60D3
:105246002A9001FDE0FCA3E0FDA3E0FEA3E0FF7BC6
:10525600FF7AFF79FF78FFEF2BFFEE3AFEED39FD7F
:10526600EC38FC9001FD12202880BFC298AF99EF60
:1052760012208552CB6152D76252E36352EB6452DD
:10528600F765530366530F67531B685327695333F8
:105296006A533F6B534B6C53576D53636E53716F29
:1052A600537D7053917153997253A77353B57453C9
:1052B600FA75540876541677542478543279544043
:1052C6007A0000544D900022E0FEA3E0FF126B9599
:1052D60022900024E0FEA3E0FF126B9522AF4BAEB6
:1052E6004A126B9522900028E0FEA3E0FF126B9510
:1052F6002290002AE0FEA3E0FF126B952290002C7C
:10530600E0FEA3E0FF126B952290002EE0FEA3E0E4
:10531600FF126B9522900030E0FEA3E0FF126B9522
:1053260022900032E0FEA3E0FF126B95229000343B
:10533600E0FEA3E0FF126B9522900036E0FEA3E0AC
:10534600FF126B9522900038E0FEA3E0FF126B95EA
:105356002290003AE0FEA3E0FF126B9522E50D24B1
:1053660088FFE50C3413FE126B95229001FBE0FEDC
:10537600A3E0FF126B95229001F9E0FEA3E0FFEF98
:105386002484FFEE3403FE126B9522AF6FAE6E12CD
:105396006B9522E56B2484FFE56A3403FE126B9558
:1053A60022E50B2484FFE50A3403FE126B9522A244
:1053B6000FE433FFEF3395E0FEEFC4F8540FC868EF
:1053C600FFEEC454F048FEE5A0C4540FFD7C00EF88
:1053D6002DFDEE3CFCA210E433FFEF3395E0FEEF2B
:1053E6007805C333CE33CED8F9FFED2FFFEC3EFE62
:1053F600126B9522900010E0FFEF3395E0FE126BE2
:105406009522900011E0FFEF3395E0FE126B952296
:10541600900012E0FFEF3395E0FE126B95229000AC
:1054260013E0FFEF3395E0FE126B9522900014E037
:10543600FFEF3395E0FE126B9522900015E0FFEF2B
:075446003395E0FE126B95A7
:01544D00223C
:1067E5009001EEE4F0A3E4F09001F4E4F09001F4FC
:1067F500E0FFD3EF6480948340030268819001F049
:10680500122034000186A020983E9001F0E0FCA300
:10681500E0FDA3E0FEA3E0FFEC4D4E4F602A9001A2
:10682500F0E0FCA3E0FDA3E0FEA3E0FF7BFF7AFF21
:1068350079FF78FFEF2BFFEE3AFEED39FDEC38FCE2
:106845009001F012202880BFC2989001EEE0FEA3CF
:10685500E0FF7C007D0A121ECAAD997C00EF2DFF7A
:10686500EE3CFEEF24D0FFEE34FFFE9001EEEEF09D
:10687500A3EFF09001F4E004F00267F29001EEE07E
:04688500FEA3E0FF8F
:0168890022EC
:10564A00900201122034000186A020983E900201A7
:10565A00E0FCA3E0FDA3E0FEA3E0FFEC4D4E4F60AB
:10566A002A900201E0FCA3E0FDA3E0FEA3E0FF7B99
:10567A00FF7AFF79FF78FFEF2BFFEE3AFEED39FD57
:10568A00EC38FC90020112202880BFC298AF99EF33
:10569A0012208556E36156F2625701635710645728
:1056AA001F65572E66573D67574C68575B69576A9F
:1056BA006A57796B57886C57976D57A67257AB73B1
:1056CA0057AE7457B47557C07657CC7757D87857B2
:1056DA00E47957F07A000057FB1267E5900022EE52
:1056EA00F0A3EFF01250D9221267E5900024EEF0F1
:1056FA00A3EFF01250D9221267E5900026EEF0A32C
:10570A00EFF01250D9221267E5900028EEF0A3EFCD
:10571A00F01250D9221267E590002AEEF0A3EFF0BA
:10572A001250D9221267E590002CEEF0A3EFF01286
:10573A0050D9221267E590002EEEF0A3EFF0125036
:10574A00D9221267E5900030EEF0A3EFF01250D99B
:10575A00221267E5900032EEF0A3EFF01250D92240
:10576A001267E5900034EEF0A3EFF01250D922123E
:10577A0067E5900036EEF0A3EFF01250D9221267D7
:10578A00E5900038EEF0A3EFF01250D9221267E547
:10579A0090003AEEF0A3EFF01250D922D20DD211B6
:1057AA0022D21122A20FB3920F221267E5900010A3
:1057BA00EFF0124FD5221267E5900011EFF0124F69
:1057CA00D5221267E5900012EFF0124FD522126728
:1057DA00E5900013EFF0124FD5221267E5900014FE
:1057EA00EFF0124FD5221267E5900015EFF0124F35
:0157FA00D5D9
:0157FB00228B
:10187600021C3CE86480F8E933E83360110460F048
:10188600ED33EC337009E8FCE9FDEAFEEBFF2204D8
:1018960060DED3EB9FEA9EE99DE8C2E78CF0C2F7D3
:1018A60095F0400CE8CCF8E9CDF9EACEFAEBCFFB9F
:1018B600121C0785D0F05804700320D5B3E80470D5
:1018C600075002B2D5021C4692D5EC0460F7E4CC70
:1018D600C0E0C398F8603B94186008400DD0E0FB68
:1018E600021C1EE4FBFAC9FC8028E830E406E4C9C1
:1018F600FBE4CAFCE830E305E4C9CACBFCE85407BC
:101906006010F8C3E913F9EA13FAEB13FBEC13FCC6
:10191600D8F130F52FC3E49CFCEF9BFFEE9AFEED69
:1019260099FDD0E0FBEF4E4D4C701222DB03021CFA
:1019360043EC2CFCEF33FFEE33FEED33FDED30E7E9
:10194600EB021C1EEF2BFFEE3AFEED39FDD0E0FB5D
:1019560050130BBB0003021C46ED13FDEE13FEEF06
:0819660013FFEC13FC021C1E30
:10196E00EC4D6011E8497017ED33EC3304600DE473
:10197E00FCFFFEFD22E933E8330470F8021C3C1232
:10198E001C0758046009E4CC248150062850090233
:10199E001C46284003021C43C0E0EB4A7044B98049
:1019AE0006D0E0FB021C32EF4E701CBD8008EBFF30
:1019BE00EAFEE9FD80EBE98DF0A4FEE5F0021A5790
:1019CE00E9CDF9EAFEEBFFEF89F0A4FCE5F0CE8954
:1019DE00F0A42EFFE435F0CD89F0A42DFEE435F011
:1019EE008067EF4E7005BD80D780C3EF8BF0A4AC3F
:1019FE00F0EE8BF0A42CFCE435F0F8EF8AF0A42C7A
:101A0E00E5F038FCE433CB8DF0A42CFCE5F03BF88C
:101A1E00EE8AF0A42CFCE5F038F8E433CF89F0A47C
:101A2E002CFCE5F038CF3400CE89F0A42FFFE5F082
:101A3E003EFEE433C98DF0A42EFEE5F039CD8AF0DA
:101A4E00A42FFFE5F03EFEE43DFD33D0E0FB500752
:101A5E000BBB000F021C46EC2CFCEF33FFEE33FEEB
:061A6E00ED33FD021C1E19
:101A7400021C46EC5D046005E859047003021C3C3A
:101A8400121C07580460F6EC4860F2EC7004FDFE8A
:101A9400FF22C860DB2481C85009C3986002500645
:101AA400021C439850CAF582E9294B4A7005AB825F
:101AB400021C3275F0007C1A7880C3EF9BEE9AED1D
:101AC40099400DC3EF9BFFEE9AFEED99FDE842F0BD
:101AD400DC23ACF0D0E0FFD0E0FED0E0FDAB822010
:101AE400E7101BEB60BAEC2CFCEF33FFEE33FEED9A
:101AF40033FD021C1EE803F830E705C0F075F00062
:101B0400EF2FFFEE33FEED33FD40B830E7C280AA7D
:101B140074F8CC6480CCC86480C8F582046043C384
:101B2400EB9FF5F0EA9E42F0E99D42F0E89C45F017
:101B340060305018E5825FFFE582F42B5582FB503C
:101B4400210ABA001D09B90019088016E5825BFB59
:101B5400E582F42F5582FF50090EBE00050DBD002D
:101B6400010CC3EB9FF5F0EA9E42F0E99D42F0E8D8
:0D1B74009C45F06007CC4820E701B3EC224F
:101B8100ED33EC33600A047003BD8004ECB2E7FC72
:011B91002231
:101B920075F020800E75F010800575F0087D007ECE
:101BA200007F003392D530D503121F77EC334010FB
:101BB200EF33FFEE33FEED33FDEC33FCD5F0ED22D7
:0E1BC200E5F0247EA2D513CC92E7CDCEFF2213
:101BD000EDD2E7CD33EC3392D524814006E4FFFE0D
:101BE000FDFC22FCE4CFCECDCC24E0501174FF806C
:101BF000EDC3CC13CCCD13CDCE13CECF13CF047009
:071C0000F030D5DE021F7772
:103D4500E57B24F3F582E43400F583E0057B2290DE
:103D550000F03009039000F3E475F00112206502CC
:103D65001E722002E97F2ED2028018EF540F249094
:103D7500D43440D4FF30060BEF24BFB41A005003EF
:103D85002461FFE57C6002157C057FE57F700205F7
:103D95007E30090E9000F0E475F001122065EF0207
:103DA5001EB8026E2E7403D2098003E4C209F57BA6
:103DB5009000F012207CE4F57CF57EF57FE57C60D3
:103DC500077F20123D8880F5757DFFC203C202C2C0
:103DD50004C205C207C208C20A123D54FF700D3065
:103DE50009057F00123D99AF7FAE7E22B4255FC2E3
:103DF500D5C206123D54FF24D0B40A00501A75F0FE
:103E05000A787C30D50508B6FF0106C6A426F6203B
:103E1500D5047002D20580D924CFB41A00EF50041E
:103E2500C2E5D20602408BD20380C6D20280C0D240
:103E35000480BCD2D580BAD20780B47F20123D88D9
:103E45002004077401B57C0040F1123D45FF123D89
:103E550088023DC2D20AD2088095123D45FB123D2B
:103E650045FA123D45F94A4B700679897A417BFF3F
:103E750020042EE57C602A7E008E82758300121E4A
:103E85008B60060EEE657D70F0C2D5EBC0E0EAC032
:103E9500E0E9C0E0EE1240ECD0E0F9D0E0FAD0E085
:103EA500FB121E72FF60AAEBC0E0EAC0E0E9C0E0C9
:103EB500123D88D0E02401F9D0E03400FAD0E0FBCF
:103EC500E57D0460DCD57DD98087D20480A21240CF
:103ED500CE60F7E57D700104121C51A97D600DE5EA
:103EE5007D600914F57D124176EF60F3EA30E70253
:103EF500F404C3995079EAF4257D0430E701E4041C
:103F0500F57D800D1240CE60C1EA057D257D121C30
:103F150051EA90011FF030E701E4257D04D57D04C9
:103F2500200701141240ECE4C0E012417690011F15
:103F3500E0601320E70714F0123D70802204F0D0F2
:103F4500E014C0E07F00123D70E57D6007123D671B
:103F5500157D800B300703123D67D0E0023DC2D0CE
:103F6500E00480C41240CE609EE57D04121C519091
:103F7500011FEAF0E57D20070260010424041240D8
:013F8500EC4F
:103F860074FF04C0E0124176123D70E57D20070201
:103F96006003123D67D0E0B57DE87F45123D7A901B
:103FA600011FE07F2B30E7047F2DF404C0E0123DB3
:103FB60088D0E075F00A84C0F0123D71D0E0123D61
:103FC60071023DC2791080027908C208C20A8008CF
:103FD600D2D5790A8004790AC2D5E57D047002F546
:103FE6007DE4FAFDFEFF123D45FC7B08200313121B
:103FF6003D45FD7B1030020A123D45FE123D45FF50
:104006007B20EC3382D592D55013C3E43002069F51
:10401600FFE49EFEE42003039DFDE49CFCE4CBF854
:10402600C203EC700CCFCECDCCE824F8F870F38048
:1040360017C3EF33FFEE33FEED33FDEC33FCEB330A
:10404600FB994002FB0FD8E9EB300305F8D0E0C43A
:1040560048B203C0E00AEC4D4E4F78207B0070C298
:10406600EAB57D0040BCC0E01240EED0F0D0E020C2
:104076000304C4C0E0C4B203C0F0123D71D0F0D551
:10408600F0EB023DC21220853E5F533FCA583E30D8
:104096004C3E2C423FCE4F3FD6443FD6493E454349
:1040A6003FDC553F09463F69453ED34741A9503E4F
:1040B600342D3E382E3E5B2B3E3C233E592041920A
:1040C6002A3DF44800003E53E57DB4FF03757D06A6
:1040D600123D45FC123D45FD123D45FE123D45FF94
:1040E600900118021C8E790AA2D520051430070902
:1040F600B910020404B9080104A2D520080250012F
:10410600042004689204B57C005034C0E07F20305F
:1041160005197F30A20472087207500F124145C27A
:1041260004C208C207C20A7F30800F300703E9C005
:10413600E0123D88300703D0E0F9D0E0B57CCC3002
:1041460007177F30B9100C123D887F583006077F5D
:10415600788003B90803123D883004057F2D023D9F
:10416600887F20200AF87F2B2008F322920480CF34
:104176007F00B40700500B2418F582E43401F58360
:10418600E0FF22286E756C6C2900D203123D453083
:1041960003F8C203787C30D50108F6023DF42D50B1
:1041A600434958123D452403B405004001E49041BB
:1041B600A493123D79743A123D79D205757C0402B6
:0241C6003FCAEE
:0D6ED400ED33EC3360065004EC6480FC22CA
:10673900021C3C22EDA2E7D2E7F9EC3340F260F308
:10674900B4FF08ED547F70E8021C46F82481C2E0CA
:10675900C0E0F40428FAC313FCED92E7FD9000E4CD
:10676900122028EEA2E7E9BA7F02C313340094008D
:10677900FA75F091A4E5F013F494FE8AF0A433E5D8
:10678900F033248CD313FDE492E7FE7F007C3F7540
:106799008302ECC0E0F8EDC0E0F9EEC0E0FAEFC02A
:1067A900E0FB8583F09000E4121FD085F083121A74
:1067B90077D0E0FBD0E0FAD0E0F9D0E0F812187D0C
:1067C900ED6480FD30E7011CD583C7ED33CC33F888
:0C67D900D0E0A2E71328C313CC13FD226C
:1069C9009000E41220289000E8E0F8A3E0F9A3E0A1
:1069D900FAA3E0FB9000E4E0FCA3E0FDA3E0FEA342
:1069E900E0FF121A77125B489000E4122028900009
:1069F900E8E030E7599000E4E0FCA3E0FDA3E0FE05
:106A0900A3E0FFECC0E0EDC0E0EEC0E0EFC0E0E4E1
:106A1900FFFEFDFC9000E4E0F8A3E0F9A3E0FAA38F
:106A2900E0FB121B147BDB600250087A0F7949786E
:106A39004080067A0F794978C0D0E0FFD0E0FED0D7
:106A4900E0FDD0E0FC12187D9000E41220289000AF
:0D6A5900E4E0FCA3E0FDA3E0FEA3E0FF22CB
:1059A0003A70FA83BCAAE9E43E81E0F8BF9DE9E6DB
:1059B0003F80000039283C1ABB9969663DA335E356
:1059C000BF255DE73FC90FDB418DDBCCC44936EE17
:1059D00045C9913FC5B0F83D3F800000C317F5347D
:1059E000452FFA73C60AFDDD125AA904A2E19200FE
:1059F0001420E0159059A07404121D938030125A9F
:105A0000A930E102B20020E0EBA883A9829000E473
:105A1000122028898288839059B47404121D9385BA
:105A200082F09000E4121FEC85F08212196EED4CAA
:105A30006007300004EC6480FC22125AA9C0E0A880
:105A400083A9829000E4122028898288839059D803
:105A50007403121D938582F09000E4121FEC85F010
:105A60008212196E9000E4E0CCF0A3E0CDF0A3E048
:105A7000CEF0A3E0CFF09059C87403121D93D082EA
:105A80008582F09000E4121FEC85F082E58230E020
:105A900007121A77B2008096EFCBFFEECAFEEDC96F
:105AA000FDECC8FC121A778085ED33EC547FCC33C3
:105AB000920024605007D0E0D0E0021C3C7B837A47
:105AC000F97922783E12196EEDF933ECF83324811E
:105AD0005011EFFBEEFA121BD0121B92ECB2E7FC56
:105AE00012187DED33EC33602F2403F8C313FCED63
:105AF00092E7FDE82481E4501FECF8EDF9EEFAEFAF
:105B0000FB121BD0EF04C2E0FCF582121B9CECB22E
:105B1000E7FC12187DE58203FAED33EC33600714DD
:085B200013FCED92E7FDEA22FF
:105B2800BE1249253E4CCCCDBEAAAAAB3F80000090
:105B38003E7ADBB03EED63383F24BC7D3F490FDB46
:105B4800ED33ECC2E7CC339200B4FF13ED547F6021
:105B580003021C3C7FDB7E0F7DC97C3F025C3DC29B
:105B680001C3947F401E7007EDD2E794904015EF73
:105B7800FBEEFAEDF9ECF87F007E007D807C3F12A9
:105B88001A77D201ED33EC33248430E705E4C0E022
:105B9800806B04FAEDD2E754F0C333DAFD540734CE
:105BA800002323C0E0CCC0E0F8EDC0E0F9EEC0E08F
:105BB800FAEFC0E0FBE4121B9CEC24FEFC9000EC26
:105BC80012202812196E7B007A007980783F12180B
:105BD8007D9000ECE0B2E7CCF0A3E0CDF0A3E0CEFE
:105BE800F0A3E0CFF0D0E0FBD0E0FAD0E0F9D0E0CD
:105BF800F812187D9000EC121FEC121A779000EC46
:105C0800122028905B287403121D939000EC121F39
:105C1800EC12196ED0E0600F2434F582E4345BF5A1
:105C280083121FF812187D30010B7BDB7A0F79C9BC
:105C380078BF12187DED33EC336006ECA20092E7D2
:025C4800FC223C
:106198009000E412202874FFFFFEFDFC9000E4E06C
:1061A800F8A3E0F9A3E0FAA3E0FBC3121F85603867
:1061B8007F807E967D187C4B9000E4E0F8A3E0F9A0
:1061C800A3E0FAA3E0FB121B146002501B7F807E41
:1061D800967D187CCB9000E4E0F8A3E0F9A3E0FA00
:1061E800A3E0FB121B14500F9000E4E0FCA3E0FDB9
:1061F800A3E0FEA3E0FF229000E4E0FCA3E0FDA3FF
:10620800E0FEA3E0FF121BD09000E81220289000C7
:10621800E8E0FCA3E0FDA3E0FEA3E0FFEC121B9284
:10622800C8ECC8C9EDC9CAEECACBEFCB9000E4E010
:10623800FCA3E0FDA3E0FEA3E0FF121879E4FBFA5B
:10624800F9F8121B14602640249000E8E0FCA3E053
:10625800FDA3E0FEA3E0FFEF24FFFFEE34FFFEED19
:1062680034FFFDEC34FFFC9000E81220289000E891
:10627800E0FCA3E0FDA3E0FEA3E0FFEC121B9222EA
:101C0700E9D2E7C933E833F892D5EDD2E7CD33EC23
:071C170033FC5002B2D5229C
:101C1E00EC30E7100FBF000C0EBE00080DBD000427
:101C2E000BEB6014A2D5EB13FCED92E7FD2274FFD3
:101C3E00FCFDFEFF22E480F8A2D574FF13FC7D802C
:031C4E00E480EF40
:101C5100F920E73624F950037907E4F42402FBE57F
:101C610082158270021583DBF6E024FB501BE960CC
:101C710014E4F0E582158270021583E004F0B40AE1
:0D1C810008E4F0D9EE7401F00A22C2D52269
:101C8E00ED33EC3392D5FA602AB4FF33EDC2E77B25
:101C9E00FF60067A1C79B3E4227A1C79BC20D50445
:101CAE007A1C79B7224E614E002B494E46002D49C3
:101CBE004E4600E47A08F0A3DAFC7B00740722C0DB
:101CCE0083C082ECC0E0EDC0E0EEC0E0EFC0E0EA21
:101CDE0075F010A4CAABF075F04DA42BFBE435F0F3
:101CEE00FCEA2410FAEB34C5FBEC34D9FCEDC2E768
:101CFE00FF75F056A4F42411C5F0F434C58FF0A48A
:101D0E002AE5F03BE43CF020E714121E10D0E0FF71
:101D1E00D0E0FED0E0FDD0E0FC121A778014F4047F
:101D2E00121E10D0E0FFD0E0FED0E0FDD0E0FC129D
:101D3E00196ED082D083E0FAEDD2E7CD33EC3324A6
:101D4E0082FBE4C3CF33CFCE33CECD33CD33DBF3F3
:101D5E007B0775F00A846004F0A31B0AE5F0F0A37C
:101D6E008FF0740AA4FFACF08EF0740AA42CFEACB3
:101D7E00F050010C8DF0740AA42CFDE435F0F0A3A4
:051D8E00DBDE740722FA
:101D9300C0E0EFFBEEFAEDF9ECF812196ED0E0F5C6
:101DA300F0EFFBEEFAEDF9ECF8121FDCA3A3A3A30B
:101DB300E8C0E0E9C0E0EAC0E0EBC0E0C0F012191F
:101DC3006E121FF8A3A3A3A312187DD0F0D0E0FBDB
:0D1DD300D0E0FAD0E0F9D0E0F8D5F0D4224D
:101DE0003F8000004120000042C80000447A00000B
:101DF000461C400047C35000497424004B1896808D
:101E00004CBEBC205A0E1BCA6753C21C749DC5AE83
:101E1000FB60065407601C2323121E3EEB543860FF
:101E200009121E2A121E3912196EECF8EDF9EEFA9B
:101E3000EFCB22EB121E3980F1543803241C901D85
:101E4000E0FE93FC0EEE93FD0EEE930ECE93FF227A
:10694900022245E493A3F8E493A34003F68001F2FD
:1069590008DFF48029E493A3F85407240CC8C3334F
:10696900C4540F4420C8834004F456800146F6DF1E
:10697900E4800B0102040810204080906D1FE47E22
:10698900019360BCA3FF543F30E509541FFEE49313
:10699900A360010ECF54C025E060A840B8E493A3DA
:1069A900FAE493A3F8E493A3C8C582C8CAC583CA05
:1069B900F0A3C8C582C8CAC583CADFE9DEE780BEBD
:016D6700002B
:101E5000C2D530F707B2D563F0FF05F030E70CB21A
:101E6000D5F4048463F0FF05F080018430D502F4DA
:021E700004224A
:101E7200BB010689828A83E0225002E722BBFE026E
:091E8200E32289828A83E49322A1
:101E8B00BB010CE58229F582E5833AF583E022500C
:101E9B0006E92582F8E622BBFE06E92582F8E22256
:0D1EAB00E58229F582E5833AF583E4932270
:101EB800BB010689828A83F0225002F722BBFE0109
:021EC800F32203
:101ECA00EF8DF0A4A8F0CF8CF0A428CE8DF0A42E2C
:021EDA00FE22E6
:101EDC00C2D5EC30E709B2D5E4C39DFDE49CFCEE21
:101EEC0030E715B2D5E4C39FFFE49EFE1220D8C3A1
:101EFC00E49DFDE49CFC80031220D830D507C3E49C
:061F0C009FFFE49EFE228F
:101F1200C5F0F8A3E028F0C5F0F8E582158270025A
:061F22001583E038F022F7
:101F2800E88FF0A4CC8BF0A42CFCE98EF0A42CFC58
:101F38008AF0EDA42CFCEA8EF0A4CDA8F08BF0A4D6
:101F48002DCC3825F0FDE98FF0A42CCD35F0FCEB35
:101F58008EF0A4FEA9F0EB8FF0A4CFC5F02ECD39FA
:0F1F6800FEE43CFCEAA42DCE35F0FDE43CFC2267
:106D6800C2D5E830E70FB2D5E4C39BFBE49AFAE456
:106D780099F9E498F8EC30E717B2D5126D9E122114
:106D880069E4C39BFBE49AFAE499F9E498F8800370
:106D980012216930D50DE4C39FFFE49EFEE49DFDFA
:046DA800E49CFC2249
:0E1F7700C3E49FFFE49EFEE49DFDE49CFC227B
:101F8500EB9FF5F0EA9E42F0E99D42F0E89C45F0B2
:011F95002229
:101F9600BB010789828A83021FD05005E9F8022116
:101FA600FBBBFE05E9F802220789828A83021FDC51
:101FB600BB010789828A830220285005E9F802229C
:0A1FC6002DBBFE05E9F802223922C6
:0C1FD000E0FCA3E0FDA3E0FEA3E0FF2284
:101FDC00E493FC740193FD740293FE740393FF224B
:0C1FEC00E0F8A3E0F9A3E0FAA3E0FB2278
:101FF800E493F8740193F9740293FA740393FB223F
:10200800BB010789828A83021FEC5005E9F8022286
:1020180013BBFE05E9F802222089828A83021FF891
:0C202800ECF0A3EDF0A3EEF0A3EFF0222B
:10203400A8828583F0D083D08212204B12204B12C9
:10204400204B12204BE473E493A3C583C5F0C583EE
:10205400C8C582C8F0A3C583C5F0C583C8C582C8F6
:012064002259
:10206500F8E0FBA3A3E0F925F0F0E5821582700204
:072075001583E0FA38F022A8
:09207C00EBF0A3EAF0A3E9F02265
:10208500D083D082F8E4937012740193700DA3A3EA
:1020950093F8740193F5828883E4737402936860FE
:0620A500EFA3A3A380DFFE
:1020AB00D083D082F8E4937012740193700DA3A3C4
:1020BB0093F8740193F5828883E473740293B5F0FB
:0D20CB00067403936860E9A3A3A3A380D863
:106E2E00EFB40A07740D126E39740A309811A899CE
:106E3E00B8130CC2983098FDA899C298B811F630C4
:076E4E0099FDC299F599229C
:106E6D00C3EE6480948040028007C3E49FFFE49EDC
:026E7D00FE22F3
:1020D800BC000BBE0029EF8DF084FFADF022E4CCEC
:1020E800F875F008EF2FFFEE33FEEC33FCEE9DECB5
:1020F800984005FCEE9DFE0FD5F0E9E4CEFD22EDFB
:10210800F8F5F0EE8420D21CFEADF075F008EF2F44
:10211800FFED33FD4007985006D5F0F222C398FD35
:052128000FD5F0EA22D2
:10212D0075F008758200EF2FFFEE33FECD33CDCC69
:10213D0033CCC58233C5829BED9AEC99E5829840EC
:10214D000CF582EE9BFEED9AFDEC99FC0FD5F0D6C9
:10215D00E4CEFBE4CDFAE4CCF9A88222B800C1B9F3
:10216D000059BA002DEC8BF084CFCECDFCE5F0CB31
:10217D00F97818EF2FFFEE33FEED33FDEC33FCEB6A
:10218D0033FB10D703994004EB99FB0FD8E5E4F925
:10219D00FA227818EF2FFFEE33FEED33FDEC33FC12
:1021AD00C933C910D7059BE99A4007EC9BFCE99A06
:1021BD00F90FD8E0E4C9FAE4CCFB2275F010EF2F4B
:1021CD00FFEE33FEED33FDCC33CCC833C810D7074B
:1021DD009BEC9AE899400AED9BFDEC9AFCE899F886
:0E21ED000FD5F0DAE4CDFBE4CCFAE4C8F92219
:0C21FB00E6FC08E6FD08E6FE08E6FF2210
:0C220700E2FC08E2FD08E2FE08E2FF2213
:0D221300E6FB08E6F908E6FA08E6CBF8223B
:0D222000E2FB08E2F908E2FA08E2CBF8223E
:0C222D00ECF608EDF608EEF608EFF622DD
:0C223900ECF208EDF208EEF208EFF222E1
:00000001FF
